:046EF9000100014152
:10696400AF50055074D02FF582E4341DF583E599BA
:10697400F022D3E5309400E52F94002290000FE03C
:0369840064032287
:0300030002566939
:0B566900C0E0C083C082C0D075D00834
:10567400852E82852D83E493FF201304C4540FFFE9
:10568400430FF08F80C284D28500C2870000D28786
:10569400007580FF7580FEC284C28500C287000049
:1056A400D287007580FF30130CC213052EE52E70CF
:0956B40006052D8002D213D2A8D4
:0956BD00D0D0D082D083D0E032BD
:03000B0002197661
:10197600C0E0C0F0C083C082C0D075D008758CD8D6
:10198600758A92D28C12414D12627BE531D3940056
:1019960040171531E53164056009E531640F6003D0
:1019A600021B88126BA9021B88753114E54ED3946D
:1019B600004002154EE54FD394004002154FE53A1C
:1019C600D394004002153AE54BD394004002154BE0
:1019D600154CE54C123B441B7A001B4F011B27029A
:1019E6001AFF031A7C041A63051A4A061A31071AE3
:1019F600180819FF0900001B85D3E52C9400E52B78
:101A060094005003021B88E52C152C704D152B02F3
:101A16001B88D3E5379400E53694005003021B88F3
:101A2600E537153770021536021B88D3E548940052
:101A3600E54794005003021B88E5481548700215D7
:101A460047021B88D3E54A9400E5499400500302F7
:101A56001B88E54A154A70021549021B88D3E52AF8
:101A66009400E52994005003021B88E52A152A7084
:101A7600021529021B887885E6FF7003021B88EF92
:101A8600B40105900524801BEFB40210126976405C
:101A96002FE53015307002152F021B88EFB4030CAA
:101AA600900526E0F52FA3E0F5308028EFB4041268
:101AB600126976400BE53015307002152F021B882F
:101AC6008012EF64057003021B88EFB4060C752FB5
:101AD60002753058788506021B88EF64076003029A
:101AE6001B88126976400BE53015307002152F02FF
:101AF6001B8878857600021B88D3E5399400E53883
:101B060094004008E539153970021538D3E53C9440
:101B160000E53B9400406BE53C153C7002153B80AC
:101B260061D3E5579400E55694004008E5571557EC
:101B360070021556D3E5559400E55494004043E5EC
:101B4600551555700215548039D3E5359400E534A2
:101B560094004008E535153570021534301423D34A
:101B6600E5339400E53294004018E53315337012DE
:101B76001532800EE551D39400400415518000754E
:0D1B86004C0AD0D0D082D083D0F0D0E03215
:030013000246554D
:0D465500C0E0C0F0C083C082C0D075D0109E
:10466200E545C3945040030246F52023030246F574
:10467200300C030246F5E5A0540FF5587D077F0183
:10468200124EAB5046202243E545700CE558B40C5F
:1046920007201004D210805B20032A2010277F0FEE
:1046A200126E8990000FE0FF64016004EFB403040E
:1046B2007F80800990000FE0B402057FA0120016EF
:1046C200754202D20390053CE0F53A90002BE0B52A
:1046D200580D7D087F05124EAB5004D2258014057B
:1046E2003EE53EAE3D7002053D14F5828E83E558EF
:0346F200F005458B
:0B46F500D0D0D082D083D0F0D0E032D3
:0300230002638AEB
:10638A00C0E0C083C082C0D075D018309819C298B6
:10639A00E599B40A08126964755000800AE550C389
:1063AA0094905003126964309902C299D0D0D08275
:0563BA00D083D0E032A9
:03003B000248F880
:0D48F800C0E0C0F0C083C082C0D075D018F1
:10490500C2CEE546C39410507C302479200C76AF96
:10491500A07804EF08800123D8FDF55953590F7D80
:10492500077F02124EAB5035202232E546700CE56A
:1049350059B40C07201204D212804A2004192012FF
:104945001690000FE0B4020F7F0A126E897F801265
:104955000016754202D20490053CE0F53A90002B12
:10496500E0B5590D7D087F05124EAB5004D2278066
:10497500140540E540AE3F7002053F14F5828E8375
:05498500E559F00546B4
:0B498A00D0D0D082D083D0F0D0E0323B
:104B5700E4F55AF55B755C1E755DFF855B82855ACA
:104B670083E0F55E635EFFE55EF0E0655E6003127D
:104B77006EFD635EFF855B82855A83E55EF0E065C7
:104B87005E6003126EFD055BE55B7002055AE55D2D
:104B9700155D7002155CD3E55D9400E55C940050EB
:104BA700BA75985A758921758845758DE775878017
:104BB700758CD8758AEF75C90275C808753D1E755D
:104BC7003E60753F1E7540B075B701D2A9D2E8D2D5
:0F4BD700AA75C64C75EEFF75FEFFD2AF12668849
:014BE60022AC
:026EFD0080FE15
:10694100202E0F90053AE0F54EE54ED3940040120B
:1069510080F7302E0D90053AE0F54FE54FD39400C6
:0369610050F922C8
:1068F90030300AD214900024E04420800DC2147F65
:1069090008126EBD900024E054DFF0FD7F247E0064
:04691900126354228F
:10300A008F70E57064017029202F047F018056209B
:10301A002F03023105123116400302310512311E07
:10302A00500C1231063014030231050230FB023013
:10303A00BBE57064027020202F047F028027202FB6
:10304A0003023105123126400302310512698070EC
:10305A00030231050230D5E57064036003023105CD
:10306A00202F057F03026EBD302F24123116501F08
:10307A00123126501A126980601512311E500B7FC8
:10308A000A12312E2014740230FB7F0302310230FF
:10309A002F2312313C501E7D017F02124EAB401588
:1030AA007D017F07124EAB500812310620144C8066
:1030BA00407F018043302F1712313C40127D017F3F
:1030CA0002124EAB500912698060047F02802930D7
:1030DA002F297D017F01124EAB5020126980701B8F
:1030EA007D017F07124EAB500D7F0912312E20143D
:1030FA000AD2300268F97F01126ED0227F09126E5D
:10310A00D0900536E0F532A3E0F533227D017F0148
:10311A00124EAB227D017F07124EAB227D017F0248
:10312A00124EAB22126ED0900536E0F532A3E0F5CE
:0A313A0033227D017F01124EAB220B
:104BE700C2957FFF126EBD124B577F071262B250FC
:104BF7000512003E8003126038D28C7F081262B221
:104C0700500512420D80FEC22A12681A9000D1E0A8
:104C1700FF7C117D00125BB3125D2690000FE0B49C
:104C27000105122834801090000FE0FF6402600431
:104C3700EFB40303123271123D2E301D11E542709D
:104C47000DE52754A060077FA0126E89C21D7D075E
:104C57007F05124EAB4002C200E552C3940A50BB17
:104C67003014B8E533453270B2C2301268F980AB00
:104A2E00EF253EFFEE353DCF2401FDE43FFC22AFE6
:104A3E005A7E00EF2403FDEE33FC22E53E255AF5A7
:104A4E0082E4353DF58322E540255AF582E4353F73
:104A5E00F58322E56F256DF582E4356EF583E0FF73
:104A6E00E56F256DF582E4356EF58322E55A240255
:104A7E00FFE433FE22E56C2401FFE433FEC3E56D53
:104A8E009FEE6480F874809822EF2540FFEE353F4C
:104A9E0022C2017FF47E01126BFFE56C25E0F56CFE
:104AAE00756D0122E55C2EF582E4355BF583E0FD44
:084ABE0022753D1E753E6022C9
:106BFF00EF1FAA0670011ED39400EA9400400BE425
:0A6C0F00FDEDC394C850E90D80F7B5
:016C19002258
:105142008F5BE55BB401197D017F06124EAB500CFB
:105152009000B1E0FF7C0D7D00125BB378850622E2
:10516200E55BB402131251B450439000B2E0FF7CED
:105172000D7D20125BB38035E55BB404161251B489
:10518200500C9000B4E0FF7C0D7D60125BB378851B
:10519200760622E55BB403197D027F06124EAB5000
:1051A2000C9000B3E0FF7C0D7D40125BB3788576F6
:0A51B20001227D027F06124EAB229F
:104EAB00BF0107900020E0FE8048BF020790002161
:104EBB00E0FE803EBF0307900022E0FE8034BF047B
:104ECB0007900023E0FE802ABF0507900024E0FE38
:104EDB008020BF0607900025E0FE8016BF070790D5
:104EEB000026E0FE800CBF0807900027E0FE800242
:104EFB00E4FEBD0103EE1322BD0204EEA2E122BDCE
:104F0B000304EEA2E222BD0404EEA2E322BD0504DB
:104F1B00EEA2E422BD0604EEA2E522BD0704EEA23A
:074F2B00E622BD0802EE338F
:014F3200225C
:101D9400124ABF900100E0F55A124A49E0123B444E
:101DA4001DC3011DF8021E2D031E62041E97051E8D
:101DB400CC061F01071F31081F5D0900001F871291
:101DC4004A49A3E0B40A15E55A124A7CE545B50729
:101DD4000BE4B506077D017F01021F45124A3DE56C
:101DE400456D7001EC6003021F87124A2EC2287FE2
:101DF40001021F5A124A49A3E0B40A15E55A124ACD
:101E04007CE545B5070BE4B506077D017F02021F9B
:101E140045124A3DE5456D7001EC6003021F8712CF
:101E24004A2EC2287F02021F5A124A49A3E0B40A6A
:101E340015E55A124A7CE545B5070BE4B506077D5E
:101E4400017F03021F45124A3DE5456D7001EC60B8
:101E540003021F87124A2EC2287F03021F5A124A06
:101E640049A3E0B40A15E55A124A7CE545B5070BC7
:101E7400E4B506077D017F04021F45124A3DE5458E
:101E84006D7001EC6003021F87124A2EC2287F0482
:101E9400021F5A124A49A3E0B40A15E55A124A7CB1
:101EA400E545B5070BE4B506077D017F05021F452F
:101EB400124A3DE5456D7001EC6003021F87124A2A
:101EC4002EC2287F05021F5A124A49A3E0B40A15FC
:101ED400E55A124A7CE545B5070BE4B506077D01D2
:101EE4007F06021F45124A3DE5456D7001EC600313
:101EF400021F87124A2EC2287F06021F5A124A491D
:101F0400A3E0B40A14E55A124A7CE545B5070AE48D
:101F1400B506067D017F078028124A3DE5456D70B0
:101F240001EC705F124A2EC2287F078029124A49A9
:101F3400A3E0B40A0F124A49A3A3E070077D017F0E
:101F440008024E20124A3DE5456D7001EC703412D2
:101F54004A2EC2287F0802100F124A49A3A3E07038
:101F640022124A49A3E024F96008147016E4FF021F
:101F74005EC27FF47E01126BFF7D5E7F0212665E9D
:031F840012420DF9
:011F87002237
:101B9300753F1E7540B0900108E0F55A124A55E0B2
:101BA300123B441BC5011BFD021C35031C6D041CA9
:101BB300A5051CDD061D15071D48081D7D09000030
:101BC3001D93124A55A3E0B40A13124A7AE546B5A7
:101BD300070BE4B506077D017F01021D60AF5A12B2
:101BE3004A3FE5466D7001EC6003021D93124A976C
:101BF300124A35D2287F01021D7A124A55A3E0B456
:101C03000A13124A7AE546B5070BE4B506077D01C8
:101C13007F02021D60AF5A124A3FE5466D7001EC28
:101C23006003021D93124A97124A35D2287F02029B
:101C33001D7A124A55A3E0B40A13124A7AE546B54F
:101C4300070BE4B506077D017F03021D60AF5A123F
:101C53004A3FE5466D7001EC6003021D93124A97FB
:101C6300124A35D2287F03021D7A124A55A3E0B4E3
:101C73000A13124A7AE546B5070BE4B506077D0158
:101C83007F04021D60AF5A124A3FE5466D7001ECB6
:101C93006003021D93124A97124A35D2287F040229
:101CA3001D7A124A55A3E0B40A13124A7AE546B5DF
:101CB300070BE4B506077D017F05021D60AF5A12CD
:101CC3004A3FE5466D7001EC6003021D93124A978B
:101CD300124A35D2287F05021D7A124A55A3E0B471
:101CE3000A13124A7AE546B5070BE4B506077D01E8
:101CF3007F06021D60AF5A124A3FE5466D7001EC44
:101D03006003021D93124A97124A35D2287F0602B6
:101D13001D7A124A55A3E0B40A12124A7AE546B56F
:101D2300070AE4B506067D017F078031AF5A124AE0
:101D33003FE5466D7001EC7057124A97124A35D24F
:101D4300287F078032124A55A3E0B40A13124A7A55
:101D5300E546B5070BE4B506077D017F08024E2073
:101D6300AF5A124A3FE5466D7001EC7023124A9751
:101D7300124A35D2287F0802100F124A55A3A3E056
:101D8300700E124A55A3E024F870057F01125EC25B
:011D9300222D
:0447AB008C5B8D5C3A
:1047AF00055CE55C7002055B14F5828C83E0F970A3
:1047BF0003024852EF7005124ABF8009BF01067508
:1047CF003F1E7540B0302846EF7007E9654560021F
:1047DF00C322BF0107E965466002C322E4FEEEC3B0
:1047EF00995029EF700F124AB2E53E2E124A4DE052
:1047FF006D6002C322EF6401700F124AB2E5402EC2
:10480F00124A59E06D6002C3220E80D2D3222028B3
:10481F0033E4FEEEC3995029EF700F124AB2E53E12
:10482F002E124A4DE06D6016C322EF6401700F1215
:10483F004AB2E5402E124A59E06D6002C3220E8043
:04484F00D2D322C3DB
:014853002242
:06100F008F5BAB05AA0493
:101015007D027F07124EAB5011E55BB4050C8B8248
:101025008A83E06405700302127C7D017F07124EFE
:10103500AB5011E55BB4050C8B828A83E0640670C6
:101045000302127CC229EB24FFF582EA34FFF58303
:10105500E0F55D8B828A83E0FFF55EA3E0F9F55F3D
:10106500EF123B44108501108C02109303109A0473
:1010750010A10510A80610AF0710B608000010BB98
:10108500755C01D229802F755C02D2298028755C98
:1010950004D2298021755C08D229801A755C10D28A
:1010A500298013755C20D229800C755C40D229807B
:1010B50005755C80D229E924FE700302117D24F8B0
:1010C500605C2409600302118FE55BB401059000A3
:1010D500208045E55BB40205900021803BE55BB4CB
:1010E50003059000228031E55BB404059000238060
:1010F50027E55BB40505900024801DE55BB4060576
:101105009000258013E55BB407059000268009E56E
:101115005B64087077900027E0455CF0806EE55BC6
:10112500B401059000208045E55BB40205900021DF
:10113500803BE55BB403059000228031E55BB40498
:10114500059000238027E55BB40505900024801DEC
:10115500E55BB406059000258013E55BB4070590B3
:1011650000268009E55B64087022900027E0FFE512
:101175005CF4FEEF5EF08014E55BB4050D8B828AAE
:1011850083E0FFD22E122995C229C2292029030204
:10119500127CE55BB40109900020E0FD7F208060B2
:1011A500E55BB40209900021E0FD7F218052E55BFB
:1011B500B40309900022E0FD7F228044E55BB4047E
:1011C50009900023E0FD7F238036E55BB405099097
:1011D5000024E0FD7F248028E55BB4060990002506
:1011E500E0FD7F25801AE55BB40709900026E0FD48
:1011F5007F26800CE55BB4080C900027E0FD7F2777
:101205007E00126354126D12D2AF2028047F018034
:10121500027F02126ED0A228922E126941AD5DE4C2
:10122500FF12665EAD5EE4FF12665EE55FB4010423
:101235007D388007E55FB40A077D367F0612665E56
:10124500E55BB405031264B87D077F05124EAB500C
:101255000A200007C22F7F0312300A7D017F011289
:101265004EAB4005C22F12300A7D017F02124EABF4
:071275004005C22F12300AF0
:01127C00224F
:024E20008F5BA6
:104E2200ED24FF922E126941E55B123B444E4B0189
:104E32004E50024E55034E5A044E5F054E64064EC6
:104E420069074E6E0800004E749000208021900089
:104E520021801C9000228017900023801290002451
:104E6200800D90002580089000268003900027E0A6
:104E7200F55CE55C6024755E01E4F55DE55C30E0BF
:104E820007AD5EE4FF12665EE55CC313F55C055E8A
:104E9200055DE55DC3940840E3227D187F0212663A
:084EA2005E7D537F0212665E83
:014EAA0022E5
:1062B200C2AFD284C285BF070BC28600E580A2E2CC
:1062C20092298019BF080BC28600E580A2E39229B9
:1062D200800BBF0508C28600E580139229D286D2C0
:0562E20085D2AFA229E6
:0162E7002294
:1044F300C228D22CE4FF1259927D2E7F0312665EEE
:104503007D607F0212665E7F03126EBD3023FD2045
:1045130023FDE5456407703B7E017F50124ABF8F40
:10452300828E837407F07D01E53E2D124A4DE582AC
:1045330024FFF582E58334FFF583E0F9EF2DF5825F
:10454300E43EF583E9F00DBD08DED2287F647E00EA
:10455300126BFF7F081262B25043302895D22CE4CD
:10456300FF1259927D607F0212665E7D327F0612D2
:10457300665E7D1E7F0512665EC22CE4FF125992B1
:104583007C017D507B087F507E011254DE7F081230
:1045930062B250097F327E00126BFF80F07F647E2F
:0445A30000126BFF98
:0145A70022F1
:025475008F5A4C
:10547700900138E0F55BE55A7020E55B124A7CE560
:10548700456F7001EE704F7460255BF582E4341E42
:10549700AF82F55D8F5E7F408024E55A64017036E8
:1054A700E55B124A7CE5466F7001EE702974B02502
:1054B7005BF582E4341EAF82F55D8F5E7F101200CC
:1054C70016855E82855D83E0FFA3E0FD126D768F12
:0654D7005CE4FD124F33FE
:0154DD0022AC
:024F33008D6B84
:104F350075F020EF900280123B38AF8285836E8F2B
:104F45006FE0F56CD394004060E56C9410505AE521
:104F55006B7014124AA1124A83504E124A61124FC5
:104F6500B4056D056D80EFE56B64017019124A9FFC
:104F7500124A835034124A61124FB43023028029F9
:104F8500056D056D80EAE56B6402701D124A9F127E
:104F95004A835015124A61A3E0FD1264E8302303E9
:0E4FA500024D93056D056D80E67F50126E89FA
:084FB30022A3E0FD1264E822D4
:100A5400855C82855B83A3A3E0FF855C82855B83E1
:100A6400A3222430F58274003EF583EDF0AF62EFEB
:100A74003395E0FEE55F2FF582E55E3EF583A3A3A3
:100A8400E0FF126D51AD07AF63EF3395E0FEEF2247
:100A9400A3A3E0FFE55C2404F582E4355BF583E081
:100AA40022E55F2405F582E4355EF583E022E55F07
:100AB4002405F582E4355EF583E0FFE55F2406F561
:100AC40082E4355EF583E0222431F58274003EF53C
:100AD40083EDF0AF62EF3395E0FEE55F2FF582E53D
:100AE4005E3EF583222455F582E4340AF583EFF063
:100AF400E56275F007A422E562FD3395E0FCE55F4D
:100B04002DF582E55E3CF583E0FFE55F2DF582E59A
:100B14005E3CF583228E69F56AAF68EF3395E0FE9B
:100B2400E5662FF582E5653EF58322ECFF3395E01B
:100B3400FEEF25E0FFEE33FE75F020ED123B38E5C5
:100B4400822FF582E5833EF58322A3A3A3E0FF8DE4
:100B5400828C83E5822404F582E43583F58322E5DF
:100B6400662405F582E43565F583E022E55E75F0DB
:100B740007A42454F582E4340AF58322E55E75F073
:100B840007A42451F582E4340AF5832224E0F58293
:100B9400740A3EF583E5822DF582E5833CF58322D4
:100BA400E55E75F007A42453F582E4340AF5832244
:100BB400E55F2405F582E4355EF583E0FFE55F2417
:100BC40006F582E4355EF583E022E55E75F007A460
:100BD4002452F582E4340AF58322749F2562F58257
:100BE400E43400F58322746F2562F582E43400F561
:100BF40083222450F582E4340AF58322E560240537
:100C0400F582E4355FF58322D3EF6480948022ABD0
:100C140007AA068B828A83A3A3A3E0FFEB2404F52F
:100C240082E43AF583E0FD228F828E83A3A3A3E0BE
:100C340022855F82855E83A3A322AB5DAD5AAF5C40
:100C4400AE5B2233CE33CE92E022A2E0CE13CE139B
:100C54002275F00AA42DFDE5F03CFCE56622E56072
:100C64002405F582E4355FF583E022E56275F0083A
:100C740090015822E55E75F007A42455F582E4340A
:100C84000AF583E022AB5AAD5DAF5CAE5B22EF7C2C
:100C9400002563FDEC35628D82F58322A3A3E0FF7A
:100CA400AD5A22E5662DF582E5653CF583A3A322C2
:100CB400540FF5657808AF03AE02EF08220564E52A
:100CC40064AE632225E0FFEE33FE75F020E5642276
:100CD40075F020123B38E0FEA3E0FF22E0FAA3E027
:100CE400FB780CFFAE020822E0FCA3E0FD7804FFD1
:100CF400AE040822E5632561F582E43562F58322BA
:100D0400E5662DF582E5653CF58322E5662FF582DF
:100D1400E5653EF583222480F58274023EAF82228B
:100D24002560F560E4355FF55F22856082855F8329
:0B0D3400228F828E83A3A3E0640A22BA
:02055B008F5AB5
:10055D00C229E4F542D222D22C1259927D4B7F0250
:10056D0012665E7D02E4FF12665E7D32E4FF126666
:10057D005E7D607F0212665E7D027F07124EAB507C
:10058D00057F04126EBD900528E0F536A3E0F53722
:10059D007F03126EBDE55A7006A22392288009E5ED
:1005AD005AB40104A2249228E53745367005D229A4
:1005BD00020A223028DFE55A7006A223922880090C
:1005CD00E55AB40104A22492282028EAE55A700BBA
:1005DD00755B1E755C6085455D800EE55AB401093D
:1005ED00755B1E755CB085465DE55DD3940050036B
:1005FD00020A1C855C82855B83E0640B6003020A42
:10060D0017A3E0FFB40A0AE55DB40205D229020A78
:10061D001CEF6401701E120A5EA3E0640A7015E5FA
:10062D005D6405700F120A5E120A94120A4D1231A2
:10063D0044020A1C120A5EE0B40111120A5EA3E024
:10064D00B40109120C3E121732020A1C120A5EE0A6
:10065D006401701E120A5EA3E064027015E55D640C
:10066D0005700F120A5E120A94120A4D1261610290
:10067D000A1C120A5EE06401701D120A5EA3E0649A
:10068D00037014E55DB4050F120A5E120A94FDABFA
:10069D005A1237B0020A1C120A5EE0B4011D120A8A
:1006AD005EA3E0B40415E55DD39405400EAB5AADE1
:1006BD005CAC5BAF5D122D91020A1C120A5EE06408
:1006CD0001701D120A5EA3E064057014E55DB405AA
:1006DD000F120A5E120A94FDAB5A125A84020A1CBA
:1006ED00120A5EE06401701D120A5EA3E0640670DA
:1006FD0014E55DB4050F120A5E120A94FDAB5A1291
:10070D004D06020A1C120A5EE0B4011D120A5EA318
:10071D00E0B40715E55DD39405400EAB5AAD5CAC66
:10072D005BAF5D12443D020A1C120A5EE06401706B
:10073D001D120A5EA3E064087014E55DB4050F1286
:10074D000A5E120A94FDAB5A12631E020A1C120AAB
:10075D005EE0B40215120A5EA3E0B40A0DE55DB4C5
:10076D000308AF5A1262E8020A1C120A5EE0B402D4
:10077D0016120A5EA3E0B4010EE55DB40E09120C6B
:10078D0040122ECE020A1C120A5EE0B40216120AA4
:10079D005EA3E0B4020EE55DB40709120C401252DF
:1007AD00AF020A1C120A5EE0B40215120A5EA3E043
:1007BD00B4090DE55DB40308AF5A125409020A1CC1
:1007CD00120A5EE064027019120A5EA3E0B4091108
:1007DD00E55DB4040C120A5E120CA012672D020A1C
:1007ED001C120A5EE064037021120A5EA3E0640A23
:1007FD007018E55D64057012120A5E120A94FD12FE
:10080D006D76AD5A124700020A1C120A5EE06403AF
:10081D007029120A5EA3E064017020E55DD3940592
:10082D004019120A5E120A94FD126D76855A62AB5A
:10083D005DAD5CAC5B123E0F020A1C120A5EE064F9
:10084D00037021120A5EA3E064027018E55D640571
:10085D007012120A5E120A94FD126D76AD5A125F75
:10086D0042020A1C120A5EE0B40315120A5EA3E0EE
:10087D00B4030DE55DB40308AF5A125FBE020A1C46
:10088D00120A5EE0B40318120A5EA3E0B40410E588
:10089D005DD394034009120C89124995020A1C126A
:1008AD000A5EE0B40315120A5EA3E0B4050DE55D22
:1008BD00B40308AF5A126D64020A1C120A5EE0B44A
:1008CD000316120A5EA3E0B4060EE55DB405091227
:1008DD000C40126840020A1C120A5EE06403701993
:1008ED00120A5EA3E0B40711E55DB4040C120A5EB2
:1008FD00120CA0126B6F020A1C120A5EE0B40316F2
:10090D00120A5EA3E0B4080EE55DB40409120C40B2
:10091D00126865020A1C120A5EE064057014E55D3A
:10092D00B4040F120A54A3A3E0FDAB5A121F8802A0
:10093D000A1C120A5EE0B40516120A98B40B10E5F3
:10094D005DD394054009120C8912339D020A1C12C5
:10095D000A5EE064067014E55DB4040F120A54A338
:10096D00A3E0FDAB5A12217A020A1C120A5EE0B412
:10097D000616120A98B40B10E55DD39405400912C2
:10098D000C891226AB020A1C120A5EE06409701A69
:10099D00120A5EA3E0B40A12E55DB4040D120A5EFC
:1009AD00A3A3E0FF125D6F020A1C120A5EE0640948
:1009BD007018120A5EA3E0B40110E55DB4040B12C9
:1009CD000A5E120CA01262448045120A5EE0B40960
:1009DD0017120A5EA3E0B4020FE55DD3940440083C
:1009ED00120C3E1214EB8027120A5EE06409701A95
:1009FD00120A5EA3E0B40310E55DB4040B120A5EA7
:100A0D00120CA0125CDD80078000AF5A126B8C2097
:100A1D0029030205A2C21DD22CAF5A1259927D6034
:100A2D007F0212665E7D327F0312665E7F03126E59
:0F0A3D00BD125DB77FFF126E89E47885F6C22285
:080A4C0022FD126D76AD5A2265
:081732008E5E8F5F8D608B61FC
:10173A00120C2CFFE55F2404120AA9FD1263F38F31
:10174A006274E22562F562C394005003021933E51C
:10175A006294144003021933E5616406701D120A8B
:10176A00A5B4010C120AF4120BF67401F002192F37
:10177A00120AF4120BF6E4F002192FE561640E6006
:10178A0003021851E55F240C120AA9FFB40A14E5F2
:10179A005F240D120AA9B40A0A120AF4120B86E48B
:1017AA00F08013E55F240D120AA9FD126BE3120AF9
:1017BA00F4120B86EFF0E55F240A120AA9FFB40AB5
:1017CA0014E55F240B120AA9B40A0A120AF4120BCE
:1017DA00D4E4F08013E55F240B120AA9FD126BE32F
:1017EA00120AF4120BD4EFF0E55F2409120AA9FFDA
:1017FA00640A6006EFD39409400A120AF4120BAA8B
:10180A00E4F08010E55F2409120AA9FF120AF41213
:10181A000BAAEFF0120AA5FFB40B15E55F24061216
:10182A000AA9B40B0B120AF4120B7674FFF08008A3
:10183A0012195F120B76EFF012193B120AE9120B1A
:10184A00F67401F002192FE561640A706E120AF447
:10185A00120B86E4120AF3120BD4E4F0E55F2409B2
:10186A00120AA9FF640A6006EFD39409400A120A11
:10187A00F4120BAAE4F08010E55F2409120AA9FF0A
:10188A00120AF4120BAAEFF0120AA5FFB40B15E51F
:10189A005F2406120AA9B40B0B120AF4120B76740F
:1018AA00FFF0800812195F120B76EFF012193B1243
:1018BA000AE9120BF67401F002192FE56164097046
:1018CA0068120AF4120B86E4120AF3120BD4E41219
:1018DA000AF3120BAAE4F0120AA5FFB40B15E55F8E
:1018EA002406120AA9B40B0B120AF4120B7674FF1F
:1018FA00F08013E55F2406120AA9FD126BE3120AAF
:10190A00F4120B76EFF0E55F2407120AA9FFE55FF0
:10191A002408120AA9FD126BE3120AF4120AE91248
:10192A000BF67401F0D22B8002C22BAF60126E5FED
:10193A0022E55F2407F582E4355EF583E0FFE55F83
:10194A002408F582E4355EF583E0FD126BE3E56277
:10195A0075F007A422E55F2406F582E4355EF58377
:0C196A00E0FD126BE3E56275F007A422BB
:103144008F5E8D5FE55ED3941D5003023250E55EC1
:1031540094324003023250D22CAF5F1259927D4612
:103164007F0712665EAF5E1234C574E2255EF55EBB
:10317400120B82E07021120BCEE0701B120BA4E044
:103184007015120B70E0700F120C78700A1232690D
:103194007D537F02023246123258E55E75F007A471
:1031A400120BF6E070047D3680027D387F061266CD
:1031B4005E123258120B80E0FFD394014034EF9436
:1031C40013502F7D097F0612665E120B8012326047
:1031D4007FF47E01126BFF7D0E7F0312665E7D35E8
:1031E4007F0612665E7D097F0612665E120BCE12A2
:1031F40032607FF47E01126BFF120BA4E0FF6005C6
:10320400125A35800A1232697D0F7F0312665E7D81
:10321400277F0212665E120B70E0FFF46008126CE6
:10322400841234C580077D187F0212665E7D377F65
:103234000412665E120C78FF126C841234C57D058C
:103244007F0612665EC22CAF5F025992C22BAF5F3B
:10325400126E5F227FF47E01126BFF22E0FF126C7C
:0D326400841234C5227D187F0212665E229E
:026161008D5E51
:10616300EFD3941D402AEF9432502574E22FFFE4BD
:10617300FEEEFD3395E0FCEF75F007A42450F582A5
:10618300E4340A120B97E4F00EBE07E5D22B80022B
:07619300C22BAF5E126E5F2C
:01619A0022E2
:062ECE008E5E8F5F8D6037
:102ED400D22A120C2CFFE55F2404120AC3122FF528
:102EE400C39418501C855F82855E83A3A3A3E0FF6F
:102EF400E55F2404120AC3FD126D3E7883A60780A1
:102F040006E47883F6C22A120AB2122FF5C3943C5F
:102F1400500D120AB2FD126D3E7884A6078006E4B5
:102F24007884F6C22AE55F2407120AC3FF126DF102
:102F34008F61E561D394004017E56194085011E571
:102F44005F2407120AC3FF126DF17880A60780067A
:102F540078807601C22AE55F2408120AC3FFE55F80
:102F64002409120AC3122FFE401FE5619420501950
:102F7400E55F2408120AC3FFE55F2409120AC3FDB2
:102F8400126D3E7888A607800678887601C22AE505
:102F94005F240A120AC3FFE55F240B120AC3122F2F
:102FA400FE401FE561940D5019E55F240A120AC31F
:102FB400FFE55F240B120AC3FD126D3E7881A6075C
:102FC400800678817601C22AE55F240C120AC3FFC9
:102FD400E55F240D120AC3FD126D3E7882A6073008
:102FE4002A0712577ED22B8002C22BAF60126E5F6B
:102FF40022FD1263F38F61E56122FD1263F38F6199
:06300400E561D3940022F7
:0652AF008E5E8F5F8D6032
:1052B500D22A120C2CFFE55F2404120BC512531AD7
:1052C5009418501C855F82855E83A3A3A3E0FFE548
:1052D5005F2404120BC5FD126D3E7883A607800678
:1052E500E47883F6C22A120BB412531A943C500D7B
:1052F500120BB4FD126D3E7884A6078006E478840F
:10530500F6C22A302A0712577ED22B8002C22BAF53
:0453150060126E5F55
:0B53190022FD1263F38F61E561C322E7
:106DF100120C0C4008EF6480948A5001227F00221B
:106D3E00AE05126DF1EFC454F0FDAF06126DF1EF1A
:036D4E004DFF22D4
:1062E8008F5ED22C1259927D1E7F0812665E7D2623
:1062F8007F0812665E7D527F0412665EC22A1268AB
:106308001A125C497880E6FF125A3512593CC22CA1
:06631800AF5E1259922253
:10672D008D5EEFD3940A4006EFD3940F4003EF70C4
:10673D000E90002BEFF0D22BAF5E126E5FD322C204
:08674D002BAF5E126E5FC32248
:025409008F5EB4
:10540B00D22C1259927D207F0512665E7D2E7F0372
:10541B0012665E7D527F0412665E90002BE0F55F94
:10542B00E55FB40B067D5F7F078034E55FB40C0648
:10543B007D5E7F068029E55FB40D067D0A7F0280C5
:10544B001EE55FB40E067D327F028013E55FB40F5D
:10545B00067D467F028008E55F70077D0A7F031299
:09546B00665EC22CAF5E1259927C
:015474002215
:106B6F008D5E120C0C400EEF6480948650071263FA
:0D6B7F00BFD22B8002C22BAF5E126E5F22D0
:026840008D5E6B
:10684200120C131263F3120C0C4010EF648094A12B
:106852005009900029EFF0D22B8002C22BAF5E12BA
:026862006E5F67
:016864002211
:026865008D5E46
:10686700120C131263F3120C0C4010EF648094A106
:106877005009900028EFF0D22B8002C22BAF5E1296
:026887006E5F42
:0168890022EC
:106D5100D3EF648094814008EF64809489500122CC
:036D61007F00228E
:106E0100120C0C4008EF648094A15001227F0022F3
:0814EB008E5E8F5F8D608B6146
:1014F300120C2C14F56374FC2561F5616403600F11
:10150300E56164076009E561640B60030216CDC3FE
:10151300E5636480948050030216CDE56364809490
:101523008840030216CDE4F562120A8B7803C333B5
:10153300CE33CED8F92430F58274003EF583AF6202
:10154300EF3395E0FE120B43E4F00562E562B40865
:10155300D8756204E56164037027120AFB12172829
:10156300120A897803C333CE33CED8F9120A6678C8
:1015730003C333CE33CED8F92431F5827400021677
:10158300C4E5616407705D120AFB121728120A8909
:101593007803C333CE33CED8F9120A667803C33344
:1015A300CE33CED8F9120ACCA3120A827803C333FE
:1015B300CE33CED8F91216D5C333CE33CED8F924D1
:1015C30033F5827400120AD2E5822406120B5B12F1
:1015D3000A847803C333CE33CED8F92434F5827426
:1015E300000216C4E561640B60030216CD120AFB08
:1015F300A3E0FD1263F3126E01120A897803C33369
:10160300CE33CED8F9120A667803C333CE33CED89D
:10161300F9120ACCA3120A827803C333CE33CED88D
:10162300F91216D5C333CE33CED8F92433F58274E9
:1016330000120AD2E5822406120B5B120A84780395
:10164300C333CE33CED8F92434F5827400120AD2D0
:10165300E5822407120B5B120A847803C333CE336B
:10166300CED8F92435F58274003EF583EDF0E562BA
:10167300FD3395E0FC120B0EE5822408F582E43578
:1016830083120B0AE5822409120B5BE0FD1263F35C
:10169300126E01120A897803C333CE33CED8F924EC
:1016A30036F5827400120AD2E582240A120B5B1209
:1016B3000A847803C333CE33CED8F92437F5827442
:1016C300003EF583EDF0D22B8002C22BAF60126E89
:0116D3005FB7
:1016D400222432F58274003EF583EDF0E562FD3399
:1016E40095E0FCE55F2DF582E55E3CF583E582241B
:1016F40004F582E43583F583E0FFE55F2DF582E5AB
:101704005E3CF583E5822405F582E43583F583E0C8
:10171400FD1263F3126E01AD07AF63EF3395E0FE84
:0E172400EF780322A3E0FD1263F3126E0122A0
:045CDD008D5EAC0725
:105CE100D3EC648094804035EC64809489502EE438
:105CF100FDECFF3395E0FEEF7803C333CE33CED80E
:105D0100F92428F58274003EF583EDFF3395E0FE1A
:105D1100120B43E4F00DBD08D8D22B8002C22BAF89
:045D21005E126E5F41
:015D2500225B
:106244008D5E120C0C402FEF648094895028EF145B
:10625400FFE55E24FF922A124FBBD22CAF5E125987
:10626400927542017F327E00126BFFE54270FCC2E0
:076274002CAF5E12599222CB
:08443D008F5E8C5F8D608B61C6
:10444500856082855F83120B4EE0FD1263F38F62F8
:10445500E562D3940050030244EBE56294324003D5
:104465000244EBE55E64067036D22CAF61125992B8
:104475007D527F0512665EAF621234C5120C62B4BE
:10448500010A120BDE7401F07D388007120BDEE4A1
:10449500F07D367F0612665EC22CAF61025992E549
:1044A500602406120C66640B703C120C62B40108A1
:1044B500120BDE7401F08005120BDEE4F074F925B1
:1044C5005EF55E75F004123A7EAFF0EF7014E560AC
:1044D5002406FBE4355FFAAD62E4FF1236BBD22B4E
:0D44E5008006C22B8002C22BAF61126E5FF9
:0144F20022A7
:082D91008F5E8C5F8D608B6189
:102D9900856082855F83120B4EE0FD1263F38F62BB
:102DA900E562D394005003022EC6E56294284003DD
:102DB900022EC6E55E64067037D22CAF61125992B5
:102DC9007D527F0512665EAF621234C5120C00E0B7
:102DD900B4010A120BEA7401F07D388007120BEA7C
:102DE900E4F07D367F0612665EC22CAF610259920D
:102DF900E5602406120C04E0640B6003022EC6127F
:102E09000C00E0B40108120BEA7401F08005120B02
:102E1900EAE4F0E4FFFEE5602407120C04E5822EE3
:102E2900120B5BE0B40B04AF0680040EBE08E7EF9B
:102E39007003022EC6C394084003022EC6120C6FFB
:102E4900123B38EFF07E01EF2401FDE433FCEEC3C1
:102E59009DEC6480F87480985020E5602406120C7B
:102E690004E5822E120B5BE0FD120C6F123B38E574
:102E7900822E120B5BEDF00E80CDE5602408120C5A
:102E890004E5822F120B5BE0640B602DEF2408FE32
:102E9900C3E55E9EF55E75F004123A7EAEF0EE7003
:102EA9001CE5602407FDE4355FFC7E00ED2FFBEE99
:102EB9003CFAAD627F011236BBD22B8002C22BAF26
:042EC90061126E5FC5
:012ECD0022E2
:0836BB008F638D648A658B6644
:1036C300756801E4F567120B1DE0FF64097037129A
:1036D30037A18003120C47D8FB120B1912379378CA
:1036E30008EF088003120C47D8FB8E69F56AE5687A
:1036F300FD3395E0FC120CA7E0FF120CA7A3E0FD3D
:10370300126D76023750120B1DE0FF1237A18003B2
:10371300120C47D8FB120B191237937804EF088069
:1037230003120C47D8FB120B19A3A3E0FF126EB3CD
:10373300EF426AAE69AF6A7804EF088003120C4760
:10374300D8FB120B19A3A3A3E0FF126EB3EF426AD7
:10375300E563700DAF67120A8D120CC8900AC08022
:1037630010E563B40115AF67120A8D120CC89005FA
:1037730030120B40E569F0A3E56AF074042568F59F
:0F378300680567C3E5676480949050030236C9F8
:1037920022A3E0FF126EB3EF426AAE69AF6A221251
:0E37A2006EB37569008F6AAE697804EF082275
:0A6EB300EFD3940940037F00222270
:0237B0008B5E2E
:1037B2001263F38F61E561D394005003023899E5F7
:1037C2006194334003023899D22CAF5E1259927D34
:1037D200527F0512665EAF611234C5746F256112A5
:1037E2000BEEE060047D3880027D367F0612665E55
:1037F2007F2C7E01126BFFE561120C71123B38E0E7
:10380200F55F70077D1B7F0612665E7D577F021291
:10381200665EE55F603F756001AF5F120A8D24014D
:10382200FFE43EFEAD60ED3395E0FCC3ED9FEE6438
:1038320080F8EC648098501DAF60EF3395E0FE7520
:10384200F008E561900158120B40E0FDE4FF1266BA
:103852005E056080C47F2C7E01126BFFE5619005DE
:1038620030120CD4900000EEF0A3EFF04E70077D02
:103872001B7F0612665E7D0C7F0312665E9000005F
:10388200E07002A3E06009E56114FD7F01122AF3F2
:0E389200C22CAF5E025992C22BAF5E126E5F67
:0138A0002205
:024D06008B5EC2
:104D08001263F38F5FE55FD394004077E55F9433D8
:104D18005071D22CAF5E1259927D527F0512665E99
:104D2800AF5F1234C5749F255F120BE2E060047D0B
:104D38003880027D367F0612665E7F2C7E01126BFC
:104D4800FF7F2C7E01126BFFE55F900AC0120CD426
:104D5800900000EEF0A3EFF04E70077D1B7F061267
:104D6800665E7D0C7F0312665E900000E07002A311
:104D7800E06009E55F14FDE4FF122AF3C22CAF5E80
:0A4D8800025992C22BAF5E126E5F5B
:014D920022FE
:02631E008B5E94
:106320001263F3AD07EDD394004021ED9433501C7C
:10633000E4FC900AC0120B2FE4F0A3F00CBC10F2A6
:10634000749F2D120BE2E4F0D22B8002C22BAF5EC1
:03635000126E5F6B
:016353002227
:025A84008B5E37
:105A86001263F3AD07EDD394004038ED94335033F1
:105A9600E4FC900530120B2FE4F0A3F00CBC10F2DE
:105AA600746F2D120BEEE4F0FCECFF3395E0FE75FF
:105AB600F008ED900158120B40E4F00CBC08EAD255
:0A5AC6002B8002C22BAF5E126E5F50
:015AD00022B3
:042AF3008F628D63FE
:102AF700E4F564E5627052AF64120A8D25E0FDEEDD
:102B070033FCAF63120A8D7805C333CE33CED8F9C1
:102B1700120B90120CE08003120C4ED8FB120CB46F
:102B27008003120C4ED8FB540FF566AF63120A8D63
:102B37007805C333CE33CED8F9120B90120CEC8044
:102B470003120C4ED8FB022BB1E56264017064AF2F
:102B570064120A8D25E0FDEE33FCAF63120A8D780F
:102B670005C333CE33CED8F92450F5827405120B42
:102B770096120CE08003120C4ED8FB120CB48003A3
:102B8700120C4ED8FB540FF566AF63120A8D780509
:102B9700C333CE33CED8F92450F5827405120B9681
:102BA700120CEC8003120C4ED8FB540FF567ED5452
:102BB7000FF568E565700CE5667008E5677004E574
:102BC70068607CAD65E4FF12665EAD66E4FF126681
:102BD7005EE56564097045856769AF69FE7804EF4E
:102BE700088003120C47D8FBF569E5684269E56977
:102BF700B4990B7D09E4FF12665E7D098027E569BC
:102C070075F00A84F56AFDE4FF12665EE56A75F001
:102C17000AA4FFC3E5699FF56AFD8009AD67E4FF74
:102C270012665EAD68E4FF12665E7FF47E01126B8A
:0F2C3700FF0564C3E564648094A05003022AFA89
:012C4600226B
:1063F300EFD394004015EF940B5010EFC3940A5061
:1064030008EF75F00AA4FE8002E4FEEDD394004089
:106413000EED940B5009EDC3940A5003ED2EFEAF1D
:016423000672
:016424002255
:064995008E5E8F5F8B6057
:10499B00756105756240D3ED64809484407CED6451
:1049AB008094A55075ED24FDF563D39404406BE51D
:1049BB006320E06613F5640562E562AE6170020583
:1049CB006114F5828E83E564F07403255FF55FE473
:1049DB00355EF55EE4F563E563C395645033855F3F
:1049EB0082855E83E0FFA3E0FD126D760562E562D2
:1049FB00AC617002056114F5828C83EFF0055FE505
:104A0B005F7002055E055FE55F7002055E05638002
:104A1B00C6D22BAF60126E5FD322C22BAF60126E69
:024A2B005FC367
:014A2D002266
:043E0F008C5F8D60D7
:103E1300120C0C5003023EE7EF64809495400302BA
:103E23003EE7EB648094875003023EE7EB648094A3
:103E3300E44003023EE7120A8D7805C333CE33CE46
:103E4300D8F9120D1AF5638F64EB24FBF565D3944F
:103E5300025003023EE7E56575F00384E5F0600375
:103E6300023EE7E56575F00384F567C3941050746B
:103E7300120CC17002056314F5828E83E567F0743A
:103E830005120D24E4F565E565C395675052120DDF
:103E93002EE0F566B40A10120CC17002056314F526
:103EA300828E83E4F0800F120CC17002056314F557
:103EB300828E83E566F0120D2EA3E0FF120D2EA372
:103EC300A3E0FD126D768F66120CC17002056314B8
:103ED300F5828E83E566F07403120D24056580A7D1
:0B3EE300D22B8002C22BAF62126E5F78
:013EEE0022B1
:0826AB008E5E8F5F8D608B6174
:1026B300C22A120D35600302274812282350030251
:1026C3002743E5649408E56394075074C3E56064A5
:1026D30080948A506B120C35A3E0F562B401069026
:1026E3000520022798E562B4020690052202279886
:1026F300E562B40306900524022798E562B4040654
:10270300900526022798E562B4050690052802275E
:1027130098E562B4060690052A022798E562B40795
:102723000690052C022798E562B4080590052E80D3
:1027330064E562B40905900530805AD22A02281450
:10274300D22A022814120C35E064017052AD60AF36
:102753005FAE5E1228235003022814E5649408E553
:102763006394074003022814C3E5606480948A409D
:1027730003022814120C35A3E0F562B40A05900590
:10278300328012E562B401059005348008E562B435
:102793000209900536E563F0A3806FD22A80721296
:1027A3000C35E06402706AAD60AF5FAE5E125B1D14
:1027B3007563008F64C3E5649463E56394005051CB
:1027C300C3E560648094885048120C35A3E0F56239
:1027D300B40107900538EFF08037E562B402059045
:1027E30005398026E562B4030590053A801CE5624D
:1027F300B4040590053B8012E562B4050590053CE1
:102803008008E562B4060890053DE564F08002D2D5
:0F2813002A302A04C22B8002D22BAF61126E5FD3
:10282200221248548E638F64D3E564943BE563942B
:02283200002282
:064854008E658F66A905C8
:10485A007D057C00120D04E0C3940A4005120D0484
:10486A00E4F00DBD00010CED640A4C70E7B90607CF
:10487A00120B63FF7E0022E964077010120B637546
:10488A00F00AA4ACF0FDE5662406801BE964087012
:10489A0021120B6375F064A4ACF0FDE566240612E0
:1048AA000B67120C552407120B672DFDE43CAF056C
:1048BA00FE22E964097033120B63FF7E007C037DDC
:1048CA00E8123AA0AC06AD07E5662406120B677536
:1048DA00F064120C582407120B67120C55240812A4
:0D48EA000B672DFDE43CFEAF0522E4FEFF50
:0148F700229E
:065B1D008E658F66A905EC
:105B23007F057E00120D0FE0C3940A4005120D0F8E
:105B3300E4F00FBF00010EEF64084E70E7E964075D
:105B43007020E5662405F582E43565F583E075F09C
:105B53000AA4FFE5662406F582E43565F583E02FA4
:045B6300FF227F009E
:015B6700221B
:08339D008E5E8F5F8D608B6175
:1033A500C22AD3E56064809484500302344BE560FF
:1033B5006480948D400302344B120D356003023452
:1033C5004B120C2C123B4433EB0133F60234010350
:1033D500340B04341505341F0634290734330834F7
:1033E5003D0900003447756201756300D22A023435
:1033F50082756201756308D22A023482756201758D
:103405006310D22A8077756201756318D22A806DA0
:10341500756201756320D22A806375620175632820
:10342500D22A8059756201756330D22A804F756240
:1034350001756338D22A8045756201756340D22AC9
:10344500803BC22A8037D3E56064809484402EE5B2
:10345500606480948D5026855F82855E83A3A3E09A
:10346500B4011A855F82855E83A3A3A3E024F67069
:103475000A756201756358D22A8002C22A302A3839
:10348500E4FF120C92E4F00FBF08F7E56024FB851A
:103495006382856283F07F01E55F2404F582E4356C
:1034A5005EF583E5822F120B5BE0FE120C92EEF0C7
:0F34B5000FBF08E4D22B8002C22BAF61126E5FF3
:0134C40022E5
:044700008F5E8D5FDC
:10470400E55ED3940050030247A3E55E941540038D
:104714000247A3D22CAF5F1259927D5F7F051266C8
:104724005EAD5EE4FF12665E7D527F0412665E7FBC
:10473400F47E01126BFF75F020E55E900280123B5F
:1047440038AF828583628F63E0F560603DD3940067
:104754004046E56094105040E56025E0F5607561E1
:1047640001E5602401FFE433FEC3E5619FEE64804C
:10477400F87480985022120CF8E0FF120CF8A3E0B1
:10478400FD1264E80561056180D77D1B7F06126612
:104794005E7D5F7F0512665EC22CAF5F025992C2D6
:0647A4002BAF5F126E5FF7
:0147AA0022EC
:10217A008F5E8D5F8B60E55E640A7074E55FC39461
:10218A000A40030222E712231DE4FDFF12665EAD38
:10219A005F1222F6E55F123B4421C20121C80221E7
:1021AA00CE0321D40421DA0521E00621E60721EC39
:1021BA000821F209000021F790052002224190052A
:1021CA002202224190052402224190052602224140
:1021DA0090052802224190052A02224190052C02EC
:1021EA00224190052E022241900530804A0222E0C7
:1021FA00E55E64017052E55FD394004006E55F94A2
:10220A00034006E55F640A703C12231DE55FB40AC9
:10221A000A7D0A1222F6900532801CE55FB4010A93
:10222A007D0B122303900534800DE55FB402137D04
:10223A000C122303900536E0FEA3E0FF1264570256
:10224A0022EE0222E00222E7E55E64026003022235
:10225A00EEE55FD3940050030222E7E55F9407504E
:10226A007CD22CAF601259927D277F0812665E7D60
:10227A0006E4FF12665E7D14E4FF12665EE55F24E3
:10228A00FE601A14602114602814602F146036242A
:10229A000570437D0112231090053880307D0212AB
:1022AA00231090053980267D0312233390053A8046
:1022BA001C7D0412233390053B80127D05122340B6
:1022CA0090053C80087D0612234090053DE0FF7E84
:1022DA0000126488800EAF60126B8C8007C22BAF2D
:1022EA0060126E5FC22CAF6012599222E4FF12662E
:1022FA005E7D527F0412665E22E4FF12665E7D52A4
:10230A007F0412665E22E4FF12665E7D527F04122B
:10231A00665E22D22CAF601259927D277F08126620
:10232A005E7D06E4FF12665E22E4FF12665E7D525F
:10233A007F0412665E22E4FF12665E7D527F0412FB
:03234A00665E22AA
:044AC6008E638F6408
:104ACA000564E5647002056314F5828E83E0F56679
:104ADA00607AC3940850757F2C7E01126BFFE4F54F
:104AEA0065E565C395665064856482856383E012D3
:104AFA003B444B37004B150A4B190B4B1F0C4B25EC
:104B0A000D4B2B0E4B310F00004B3DE4FD802D7DEC
:104B1A005F7F0780287D5E7F0680227D0A7F028074
:104B2A001C7D327F0280167D467F0280107D0A7FBF
:104B3A0003800A856482856383E0FDE4FF12665E72
:0C4B4A000564E564700205630565809554
:014B5600223C
:061F88008F5E8D5F8B608F
:101F8E00C22AE55E640A600302207CE55F123B44D0
:101F9E001FBD011FD0021FE3031FF60420090520F9
:101FAE001F06203507204B082060090000207812FC
:101FBE0020B17D011220FF756101756200D22A02E7
:101FCE0020981220B17D021220FF75610175620802
:101FDE00D22A0220981220CD7D0312210C756101A8
:101FEE00756210D22A0220981220CD7D0412210C87
:101FFE00756101756218D22A0220981220E9122109
:10200E005F7D0512212F756101756220D22A022093
:10201E00981220E912215F7D0612212F756101753C
:10202E006228D22A0220981221191221737D0712DA
:10203E00213C756101756230D22A02209812211955
:10204E001221737D0812213C756101756238D22A06
:10205E008038122149E4FDFF12665E7D0912216669
:10206E00756101756240D22A8020C22A801CE55E0D
:10207E0064017016E55F24F670101221497D0A1274
:10208E002166756101756258D22A302A09AF62AE97
:10209E0061124AC68005AF60126B8CC22CAF601203
:0220AE00599245
:1020B00022D22CAF601259927D577F0212665E7D4C
:1020C00005E4FF12665EE4FDFF12665E22D22CAFCD
:1020D000601259927D577F0212665E7D05E4FF1201
:1020E000665EE4FDFF12665E22D22CAF601259924A
:1020F0007D577F0212665E7D05E4FF12665E22E474
:10210000FF12665E7D527F0412665E22E4FF126655
:102110005E7D527F0412665E22D22CAF601259920D
:102120007D577F0212665E7D05E4FF12665E22E443
:10213000FF12665E7D527F0412665E22E4FF126625
:102140005E7D527F0412665E22D22CAF60125992DD
:102150007D577F0212665E7D05E4FF12665E22E413
:10216000FDFF12665E22E4FF12665E7D527F04125E
:0A217000665E22E4FDFF12665E22A7
:1034C5008F72E572D3945940107D5A1235AC24A6FB
:1034D500FD70030235AB0235A6E572D3944F401655
:1034E500E572945A50107D501235AC24B0FD70032E
:1034F5000235AB0235A6E572D394454016E57294C4
:103505005050107D461235B424BAFD70030235AB18
:103515000235A6E572D3943B4012E5729446500CF1
:103525007D3C1235B424C4FD607C8075E572D3946E
:10353500314012E572943C500C7D321235BC24CEDC
:10354500FD6063805CE572D394274012E572943286
:10355500500C7D281235BC24D8FD604A8043E572A5
:10356500D3941D4016E572942850107D1EE4FF1279
:10357500665EE57224E2FD602D8026E572D3941324
:103585004016E572941E50107D14E4FF12665EE548
:103595007224ECFD60108009E572C394145007ADE8
:1035A50072E4FF12665E22E4FF12665EE57222E4B3
:0F35B500FF12665EE57222E4FF12665EE5722287
:105992008F6AE56A700C302C097F01126ED07FC0CD
:1059A200801FE56A700C202C097F01126EBD7FC03A
:1059B2008026E56AB40112302C0F7F02126ED07F6E
:1059C20030120016C22E026941E56AB40114202C7D
:1059D200117F02126EBD7F30126E897FC87E001267
:0359E2006BFF2236
:10691D008F69D22C1259927D607F0212665E7D3294
:10692D007F0612665E7D1E7F0512665EC22CAF6904
:04693D001259922237
:106B8C008F69D22C1259927D607F0212665E7D3025
:0D6B9C007F0312665EC22CAF69125992226F
:0E6E5F008F68302B0302691DAF68126B8C2206
:105D6F00EF24FE60101460162402701C7F01126E67
:105D7F00D07F8080107F02126ED07F2080077F033C
:105D8F00126ED07FA01200167FF47E01126BFF758A
:105D9F004204E54270FC7F647E00126BFF7F0312AA
:085DAF006EBD7FA0126E892277
:106488008E618F627C007D0A123AB2AD07E4FF127A
:10649800665E7D5B7F0612665EAE61AF627C007DE4
:1064A8000A123AB2E4FF12665E7D4A7F0702665E10
:046457008E618F6261
:10645B007C007D3C123AB21234C57D057F06126674
:10646B005EAE61AF627C007D3C123AB2ED4C600CCB
:0C647B00AF051234C57D4A7F0712665E33
:0164870022F2
:025F42008D5E72
:105F4400120C0C402FEF648094955028120A8D781F
:105F540005C333CE33CED8F9120D1AFEE4FD0FEF8C
:105F6400AA0670010E14F5828A83E4F00DBD20EEBA
:0B5F7400D22B8002C22BAF5E126E5FCA
:015F7F0022FF
:105FBE008F5E900540E0D394024015D22C12599278
:105FCE007542037F327E00126BFFE54270FC801536
:105FDE00D22CAF5E1259927D1B7F0612665E7D0C2F
:0D5FEE007F0312665EC22CAF5E1259922234
:106D64007E10900540E4F0A3DEFC7E10D22B126E60
:016D74005FBF
:016D750022FB
:106D7600BF0A02E4FFBD0A02E4FDEF75F00AA42D86
:026D8600FF22EA
:106BE300EFD394094002E4FFEDD394094002E4FD9E
:0C6BF3007804EF08800123D8FD4DFF223C
:103FC20007010203040506070707060504030201A9
:103FD20003010A0A030307050303020503020A0A8F
:103FE20004050A0A0104050A0A0A04050A0A020368
:103FF200070A0A03040A0A04024B00020032072ECF
:1040020003024B0002003202055F000302055F005B
:104012000402055F000502055F000604072E08265C
:104022000640033204072E08260640025304081EE7
:1040320008260452010008024B00020032072E0833
:104042001E08260452010003072B02350636030719
:104052002B0235063803072B0235072603072B02EE
:1040620035025302055F000F02055F001002055F73
:10407200001102055F001202055F001302055F00D6
:0A40820014080C0A1D020500241B9F
:105236007461F0A37420F0A37452F0A37401F0A378
:1052460022A3F0A37461F0A37440F022F0A37403C8
:10525600F0E4A3F0A37410F0A37403F0E4A3F0A3A6
:10526600227461F0A37441F0A3227461F0A3F0A349
:105276007430F0A3227496F0A37432F0A37495F000
:10528600A3741EF0A322F0A37461F0A314F0A37418
:1052960070F0A3E4F022A3F0A37452F0A3223CF52D
:0952A60083E0FEEF3395E0FC22E9
:10003E007E3F7FC27C017D507B081260B07E3F7F89
:10004E00CA7C017D587B081260B07E3F7FD27C0156
:10005E007D007B041260B07E3F7FDE7C017D087BDD
:10006E00041260B07E3F7FDA7C017D107B0412604B
:10007E00B07E3F7FD67C017D187B041260B07E3F40
:10008E007FE77C017D207B051260B07E3F7FE27CA6
:10009E00017D287B051260B07E3F7FEC7C017D30B8
:1000AE007B051260B07E3F7FF17C017D387B0412B0
:1000BE0060B07E3F7FF57C017D407B041260B07E98
:1000CE003F7FF97C027DA07B091260B07E407F02EB
:1000DE007C027DC07B071260B07E407F097C027D72
:1000EE00E07B051260B07E407F0E7C037D007B05B9
:1000FE001260B07E407F137C037D207B051260B0C2
:10010E007E407F187C037D407B051260B07E407F71
:10011E001D7C037D607B091260B07E407F267C03D0
:10012E007D807B091260B07E407F2F7C037DA07B9B
:10013E00091260B07E407F387C037DC07B11126057
:10014E00B07E407F497C037DE07B071260B07E402D
:10015E007F507C047D007B071260B07E407F577C11
:10016E00047D207B071260B07E407F5E7C047D4064
:10017E007B071260B07E407F657C047D607B05123C
:10018E0060B07E407F6A7C047D807B051260B07E0D
:10019E00407F6F7C047DA07B051260B07E407F7433
:1001AE007C047DC07B051260B07E407F797C047D2F
:1001BE00E07B051260B07E407F7E7C057D007B0576
:1001CE001260B07E407F837C057D407B091260B05B
:1001DE009000297417F07F031263BF9000287419E2
:1001EE00F090002074B1F09000217491F0900022F4
:1001FE007403F0900023747FF090002404F09000BC
:10020E00257403F0E4900026F0900027F090003063
:10021E0074091252527415F0A37403F0A3741512DC
:10022E0052527409F0A37403F0E4FFEFFD3395E02E
:10023E00FC74302DF58274001252A474102DF582C8
:10024E0074003CF583EEF00FBF08E0E4FFEFFD33E2
:10025E0095E0FC74382DF58274001252A474182D9A
:10026E00F58274003CF583EEF00FBF08E090052098
:10027E00E4F0A374B4F0900522E4F0A374B4F0900B
:10028E0005247401F0A374E0F0900526E4F0A37445
:10029E0078F09005287402F0A37458F090052AE4C3
:1002AE00F0A3743CF090052C7402F0A37458F07413
:1002BE000790052EF0A3F0900530F0A3F0900532D4
:1002CE00F0A3F0900534F0A3F0900536E4F0A3749B
:1002DE003CF0900538740AF09005397428F09005BA
:1002EE003A7405F090053B740AF090053CF09005C9
:1002FE003D7428F09000A47401F0900B607415F01A
:10030E00A37411F09000A57401F0900B807415F099
:10031E00A37410F09000A67401F0900BA07415F069
:10032E00A37421F09000A77401F0900BC07415F027
:10033E00A37420F09000A87401F0900BE07415F0F7
:10034E00A37431F09000A97401F0900C007415F0B4
:10035E00A37430F09000AA7401F0900C207415F084
:10036E00A37441F09000AB7401F0900C407415F042
:10037E00A37440F09000AC7401F0900C60745312B2
:10038E00524074361252407438F0A3E4F0A3745302
:10039E00F0A3E4F09000AD04F0900C807453125270
:1003AE00407434F0A37421F0A37453F0A3E4F090DE
:1003BE0000AF04F0900CC012523E7430F074031271
:1003CE00529CE4F09000B004F0900CE012523E7497
:1003DE0030F0740412529CE4F09000B104F0900DD1
:1003EE000012523674321252407452F0A37420F03E
:1003FE009000B27401F0900D201252367432F0A3B8
:10040E00740212529D7420F09000B37401F0900D9E
:10041E004074531252407433F0A3E4F09000B404CD
:10042E00F0900D601252677430F0740212524790C1
:10043E0000B57401F0900D801252677430F074059F
:10044E001252479000B67401F0900DA012526774CC
:10045E0030F0A374061252489000B77401F0900D5C
:10046E00C012526712527B7498F0A3744B1252480A
:10047E009000B87401F0900DE012526712527B7426
:10048E0093F0A374181252489000B97401F0900EB4
:10049E00001252677430F0A37413125248A3747092
:1004AE00F0A37402F09000BA14F0900E2012527065
:1004BE007412F0A374701252407461F0A314F09091
:1004CE0000BB7401F0900E40125270741112528CD7
:1004DE009000BC04F07461900E601252727414128B
:1004EE00528C9000D104F09011001252677492F069
:1004FE00A3744BF0A37490F0A37402F0A37490F065
:10050E00A37432F07499A3F0A3F0A3746012524056
:10051E0074911252407491F0A3E412524890000F5D
:10052E007401F0125DB77F01126ED07F401200167B
:10053E007D2F7F0712665E7D0C7F0312665E7D3215
:0C054E007F0612665E7D1E7F0512665E51
:01055A00227E
:0A60B0008E5A8F5B8C5C8D5D8B5E59
:1060BA00E4F9C3E55E6480F8E96480985022E9FF58
:1060CA003395E0FEE55B2FF582E55A3EF583E493CE
:1060DA00FDE55D2FF582E55C3EF583EDF00980D2A2
:0160EA002293
:10554400AF6AEF3395E0FEE56975F008A42428F509
:1055540082E43400F583E5822FF582E5833EF5830A
:10556400E0FFE56AFD3395E0FC22AB66AD65AF6410
:10557400223EF583E0FD74B82FF582741D3EF58359
:10558400EDF0056AE56A22EF3395E0FEEF25E0FFD2
:10559400EE33FE22A2E0CE13CE13223CF583EFF0CD
:0555A400056AE56A2222
:045B68008C5B8D5C69
:105B6C00EF6043D201D202D20CE4F55D855C8285F4
:105B7C005B83E0FEA3E04E6027AF5D12558BE55CC6
:105B8C002FF582E55B3EF583E0FEA3E0FF12438533
:105B9C00922820280B055DC3E55D6480949040CC71
:065BAC00C201C202C20C9E
:015BB20022D0
:045BB3008C608D6114
:105BB700EF6043D201D202D20CE4F562856182859F
:105BC7006083E0FEA3E04E6027AF6212558BE5616C
:105BD7002FF582E5603EF583E0FEA3E0FF124385E3
:105BE700922C202C0B0562C3E5626480949040CC14
:065BF700C201C202C20C53
:015BFD002285
:04438500AD07AC06CE
:10438900C22D780CEF088003125598D8FB540FF50D
:10439900637808AF05AE04EF088003125598D8FB7F
:1043A900540FF5647804AF05AE04EF088003125585
:1043B90098D8FB540FF565ED540FF566E563607108
:1043C900B4010812556E123C4D8066E563B40208CB
:1043D90012556E126AF78059E563B4030812556ED7
:1043E900123990804CE563B4040812556E126A982C
:1043F900803FE563B4050812556E1224FD8032E54D
:1044090063B4060812556E12127D8025E563B40760
:104419000812556E125AD18018E563B4080812556E
:104429006E125723800BE563B4090612556E1268A4
:034439008AA22D27
:01443C00225D
:103C4D008F678D688B69E567B40113900020E0FFE5
:103C5D0012588C900020EFF0FD7F20023D0AE567A1
:103C6D00B40211900021123D10900021EFF0FD7F64
:103C7D0021023D0AE567B40311900022123D109018
:103C8D000022EFF0FD7F22023D0AE567B40410909B
:103C9D000023123D1A900023EFF0FD7F23805EE597
:103CAD0067B40516900024123D1A900024EFF0FD24
:103CBD007F247E001263540264B8E567B406109049
:103CCD000025123D24900025EFF0FD7F25802EE587
:103CDD0067B40710900026123D24900026EFF0FDEA
:103CED007F268019E567B40819900027E0FFAB69BE
:103CFD00AD6812588C900027EFF0FD7F277E0012E3
:103D0D00635422E0FFAB69AD6812588C22E0FFAB23
:103D1D0069AD6812588C22E0FFAB69AD6812588C02
:013D2D002273
:10588C00D22EAC07BD01047E018033BD02047E0222
:10589C00802CBD03047E048025BD04047E08801E7C
:1058AC00BD05047E108017BD06047E208010BD0748
:1058BC00047E408009BD08047E808002C22EBB019C
:1058CC0005EE4204800BEB7006EEF452048002C22B
:0758DC002E302E03AF042261
:0158E30022A2
:026AF7008B67AB
:106AF900C22EEF7016ED7013E5677003025C49E56D
:0B6B090067B401077880E6FF125A35E0
:016B1400225E
:063990008F678D688B6952
:10399600E5677007123A76E4FD801AE567B4010719
:1039A600123A767D01800EE567B4020CAD69AF6808
:1039B600126E6D7D02024F33E567B40306124D9316
:1039C600C21D22E567B40415AD69AF681263F38FB3
:1039D60043754205E5427003023A7580F7E5676470
:1039E600067017E5687013F56A12554474102DF5C4
:1039F60082740012559FB408F022E56764077017B9
:103A0600E5687013F56A12554474182DF582740032
:103A160012559FB408F022E56764087027E56870C0
:103A260023E569701FF56AAF6AEF3395E0FE7410FF
:103A36002FF5827400125575B408EC754201E54203
:103A4600602D80FAE56764097025E5687021E569EF
:103A5600701DF56AAF6AEF3395E0FE74182FF58294
:0F3A66007400125575B408EC754201E54270FC0E
:093A750022AD69AF68126E6D22EA
:106A98008F67AE03AF05E567D394004012E56794AE
:106AA80007500CAD06126E6DAD07AF671266B222C5
:1024FD008F678D688B69E5677018E5687014E569FD
:10250D0070057F01126E89E569640160030226AAD8
:10251D008043E567701CE568B40117E56970057FB8
:10252D0004126E89E569640160030226AA7F040224
:10253D0026A7E5677029E56864027023E5697005D3
:10254D007F05126E89E569640160030226AA900079
:10255D000FE0B403057F010226A77F050226A7E53C
:10256D0067B4011BE5687017E56970057F02126E8F
:10257D0089E569640160030226AA7F020226A7E5A8
:10258D0067B4011CE568B40117E56970057F081291
:10259D006E89E569640160030226AA7F080226A7F9
:1025AD00E56764017029E56864027023E5697005CB
:1025BD007F0A126E89E569640160030226AA900004
:1025CD000FE0B403057F020226A77F0A0226A7E5C6
:1025DD0067B4021BE5687017E56970057F40126EE0
:1025ED0089E569640160030226AA7F400226A7E5FA
:1025FD0067B4021CE568B40117E56970057F101218
:10260D006E89E569640160030226AA7F100226A780
:10261D00E56764027024E5686402701EE569700563
:10262D007F50126E89E5696401707290000FE0B4FD
:10263D0003047F4080647F508060E567B40317E535
:10264D00687013E56970057F80126E89E569640114
:10265D00704B7F808044E567B40318E568B40113BF
:10266D00E56970057F20126E89E5696401702E7F22
:10267D00208027E56764037024E5686402701EE519
:10268D006970057FA0126E89E569B4011090000F85
:0E269D00E0B403047F8080027FA012001622AA
:10127D008F678D688B69E5677017AD69AF68126E02
:10128D006D8E348F35D3E5359400E534940050F5EB
:10129D0022E567B4011BE568B40116E5697007C264
:1012AD002F7F0112300AE569640160030214EA80A0
:1012BD0058E5676401702BE56864027025E5697077
:1012CD0007C22F7F0212300AE56964016003021420
:1012DD00EA90000FE0640370030214EAD22F7F023C
:1012ED008031E5676401702EE56864037028E56957
:1012FD007007C22F7F0312300AE569640160030293
:10130D0014EA90000FE0B40306D22F7F018004D2BF
:10131D002F7F0302300AE5676401702DE5686404D0
:10132D007027E569700CC22F7F0112300A7F4012C1
:10133D006E89E569640160030214EAD22F7F011200
:10134D00300A7F40120016807CE5676401703AE533
:10135D006864057034E569700CC22F7F0212300A83
:10136D007F10126E89E569640160030214EA900032
:10137D000FE0640370030214EAD22F7F0212300AC9
:10138D007F10120016D22E803EE5676401703BE59A
:10139D006864067035E569700CC22F7F0312300A40
:1013AD007F50126E89E569640160030214EAD22F41
:1013BD007F0312300A90000FE0B403047F408002D7
:1013CD007F50120016C22E026941E5676402702932
:1013DD00E56864017023E56970057F100214D1E59D
:1013ED0069B401057F100214DBE569640260030234
:1013FD0014EAD22E7F010214E7E56764027029E535
:10140D006864027023E56970057F200214D1E569D7
:10141D00B401057F200214DBE56964026003021448
:10142D00EAD22E7F020214E7E56764027029E568AF
:10143D0064037023E56970057F400214D1E569B43A
:10144D0001057F400214DBE569640260030214EAC2
:10145D00D22E7F030214E7E56764027023E568640A
:10146D0004701DE56970047F808059E569B401043D
:10147D007F80805AE56964027063D22E7F04805AA2
:10148D00E56764027023E5686405701DE569700405
:10149D007F048030E569B401047F048031E569641F
:1014AD0002703AD22E7F058031E5676402702EE519
:1014BD0068640670287D017F07124EAB401FE569F9
:1014CD0070057F08026EBDE569B401057F08026EE7
:0E14DD00D0E569B40207D22E7F0612299522AF
:025AD1008B67E1
:105AD300EF7037ED7034E567700690000F04802097
:105AE300E567B4010A90000F7402F0D22E801BE523
:105AF30067B40216C21D7FFF126E8990000F7403F4
:105B0300F0C22F7F0212300AD22E302E0C90000FDB
:095B1300E0FD7F0F7E00126354D7
:015B1C002266
:105723008F678D688B69E567700C125767749F2FBD
:10573300F58274008019E567B4010C125767749FF2
:105743002FF58274008016E567B4020912576F3E85
:10575300F583E4F022E567B4030912576F3EF5833E
:105763007401F022AD69AF68126E6D22AD69AF6846
:0B577300126E6D746F2FF5827400221F
:02688A008F6716
:10688C00AF057804EF08800123D8FD4BF568E56768
:10689C00B40908E568B49903025399AD68AF67125F
:0268AC0064E89E
:0168AE0022C7
:0D6E6D00EF75F00AA47C002DFFEC35F0FE5F
:016E7A0022F5
:0466B2008F688D69F7
:1066B600C3E569648094E4501BE4F56AC3E5696444
:1066C60080F8E56A648098500BC22EAF681229954F
:0466D600056A80E8E9
:0166DA00229D
:0D6E7B00C296007F051267F4126425D296BE
:016E880022E7
:106CFC00126E7BEF20E0F9C296007F061267F4C299
:066D0C00B60000D2962241
:106D1200126E7BEF20E0F9C296007F041267F4C284
:066D2200B60000D296222B
:045F80008E608F613F
:105F8400AE04AF058E638F64C296007F031267F47C
:105F9400E560FF1267F4AF611267F4E4F56212641E
:105FA40025E5642562F582E43563F583EFF0056247
:095FB400E562C3942040E7D29697
:015FBD0022C1
:085BFE008E658F668C678D68CF
:105C0600126E7BEF20E0F985656A85666BC29600A9
:105C16007F021267F4E567FF1267F4AF681267F454
:105C2600E4F569E56B2569F582E4356AF583E0FFFD
:105C36001267F40569E569C3942040E7C2B600001F
:025C4600D296F4
:015C48002239
:0A54DE008E5A8F5B8C5C8D5D8B5E37
:1054E800C2AF126CFC126E7BEF20E0F9855C608520
:1054F8005D61C296007F021267F4E55AFF1267F4F5
:10550800AF5B1267F4E4F55FAF5EEF3395E0FEC37F
:10551800E55F9FEE6480F87480985014E561255F1C
:10552800F582E43560F583E0FF1267F4055F80D803
:0B553800C2B60000D296126D12D2AF76
:015543002245
:106354008E718F728D73C2AF126CFC126E7BEF2044
:10636400E0F9C296007F021267F4E571FF1267F448
:10637400AF721267F4AF731267F4C2B60000D2961C
:06638400126D12D2AF22DF
:10603800C2AFE4F55BF55CF55DF55EF55FF55AAE6C
:106048005EAF5FAC5BAD5C125F807420255CF55C75
:10605800E4355BF55B7420255FF55FE4355EF55E3E
:0B606800055AE55AC3948940D6D2AF18
:01607300220A
:105DB700C2AF756200756300756400E4F560F56154
:105DC700F55F126CFCAE63AF64AC60AD61125BFE55
:105DD70074202561F561E43560F56074202564F56C
:105DE70064E43563F563055FE55FC3948940D312C7
:045DF7006D12D2AFA8
:015DFB002285
:10560B000500050105030507050F051F051E051CF4
:10561B00051805100201040E040A03060101040B10
:10562B000304040F020304010302040D020002022F
:10563B000300040904040305030701000303040723
:10564B00030104060402040C0516051500000615DB
:0E565B00062A060C06380633061E061206172F
:104C77002430F58274003EF583EDFF3395E0FEE5C1
:104C8700822FF582E5833EF583E0FFEDFB3395E068
:104C9700FA22AF411267F4C293126EC7D293D2AF12
:104CA700223EF583E0FC74B82FF582741D3EF58330
:104CB700ECF00D221528E528D394002225E0240BDB
:104CC700F582E43456F583E49322E4F57CD20EC2F0
:104CD70026C21CC219227FA0126E89E4F542C21DAA
:104CE70022126EC7D2B67801EF0822122C47D2CA19
:0F4CF700D20ED22622ECFF3395E0FEEF78032297
:10408C00200E2F900540E004F577D3648094815086
:10409C000302414CD3E5776480948F400375770F0E
:1040AC00900029E0FF122C4790002AE0F576124C84
:1040BC00D122301958302612124CBB400302414C0D
:1040CC00C2CAC226D21C85762822301C0A124CBBCE
:1040DC00506EC226C21C22AF7A157AEF700BC21931
:1040EC00E57625E0F528D21C22E57B30E0058576C7
:1040FC00288008E57675F003A4F528AF7B7801EFEE
:10410C0008800103D8FDF57BD226D2CA22D57708C8
:10411C00C20EE4F542C21D22057C7440257CF5825A
:10412C00E43405F583E0124CC3540FF57A74019313
:10413C00F57B700AD21CE57625E025E0F528D2192E
:01414C002250
:1050C400200E12900029E0FF122C4790002AE0F5F0
:1050D40078124CD12230195130260F124CBB505D3E
:1050E400C2CAC226D21C85782822301C0A124CBBA4
:1050F400504BC226C21C22AF7A157AEF7007C21930
:10510400C20EF54222E57B30E0058578288008E56B
:105114007875F003A4F528AF7B7801EF08800103CC
:10512400D8FDF57BD226D2CA22E543124CC3FA74C9
:0D5134000193FBEA540FF57AEBF57BD219DD
:01514100224B
:10642500E4F575D297F574C2B6126EC7AF757801EB
:10643500EF08800123D8FDF57530970343750112E8
:106445006EC7D2B60574C3E5746480948840D8AF2E
:0164550075D1
:016456002223
:096EC700000000000000000022A0
:10663200C2B7E4FEC2B6126EC7EF30E704D2B5802D
:1066420002C2B5124CE8800123D8FDFF126EC70EBC
:0B665200BE08E1C2B6D2B7D2B6D2B586
:01665D00221A
:0D001600C2AFEF4227AF27126632D2AF22F1
:0E6E8900C2AFEFF45227AF27126632D2AF220B
:1067F400E4FEC2B6126EC7EF30E704D2B58002C21F
:10680400B5124CE8800123D8FDFF126EC70EBE08F6
:05681400E1D2B6D2B58F
:01681900225C
:096ED000C2AFEF4241124C9922BD
:0A6EBD00C2AFEFF45241124C9922CB
:102C4700EF123B442CAF012CB6022CBD032CC4045D
:102C57002CCB052CD2062CD9072CE0082CE7092C05
:102C6700EE0A2CF50B2CFC0C2D030D2D0A0E2D1145
:102C77000F2D18102D1F112D26122D2D132D341445
:102C87002D3B152D42162D49172D50182D57192D4F
:102C97005E1A2D651B2D6C1C2D6E1D2D751E2D7C32
:102CA7001F2D832000002D6C75CB8E75CAC622752B
:102CB700CB9575CA772275CB9B75CA692275CBA050
:102CC70075CABA2275CBA675CA332275CBAB75CA3E
:102CD700632275CBB075CA022275CBB475CAA3221D
:102CE70075CBB875CAFA2275CBBC75CAD82275CB15
:102CF700C075CAA82275CBC475CA362275CBC775ED
:102D0700CA862275CBCA75CABC2275CBCD75CAB423
:102D17002275CBD075CA762275CBD375CA3022758A
:102D2700CBD575CAB22275CBD875CA132275CBDA43
:102D370075CA522275CBDC75CA7D2275CBDD75CA83
:102D47006E2275CBE075CA542275CBE275CA1B2279
:102D570075CBE375CAC32275CBE575CA5E2275CB01
:102D6700E675CADA22801C75CBE875CA902275CB46
:102D7700EA75CAD92275CBEC75CA092275CBED75F0
:0A2D8700CA292275CBE875CA412263
:10002600C3EF648094A15008EF25E025E0F528226F
:04003600E4F52822A3
:0235C4008F5A1C
:1035C600900118E0FFE55A7006E545D39F5012E5D5
:1035D6005A640160030236BAE546D39F50030236A9
:1035E600BAE55A7018C3E5459FF55D74602FF582FC
:1035F600E4341EAD82F55E8D5F7F40801BE55AB4D4
:103606000119C3E5469FF55D74B02FF582E4341EBB
:10361600AF82F55E8F5F7F101200167FF47E011277
:103626006BFF7D207F0512665E7D1A7F0812665E3F
:103636007FC87E00126BFFE4F55BE55BC3955D50CA
:1036460061055FE55FAE5E7002055E14F5828E83EE
:10365600E0F55C123B4436970036750A36790B3630
:103666007F0C36850D368B0E36910F0000369DE4A5
:10367600FD80277D5F7F0780227D5E7F06801C7D23
:103686000A7F0280167D327F0280107D467F02808F
:103696000A7D0A7F038004AD5CE4FF12665E055B6B
:1036A6008098E55A70047F408007E55AB401057F8B
:0436B60010126E89F7
:0136BA0022ED
:10504100200E10754406901DB8E06003D20E22E4D4
:10505100F54222E528D394004003152822C2CA153F
:1050610044E54414603D14603214601D146015144D
:105071007049901DB8E0FF7003F54222122C479051
:105081001DB9802F901DBA8015901DBBE0FF7003E4
:10509100F54222122C47901DBC8018901DBDE0FFE7
:1050A100020026901DBEE0FF7003F54222122C473C
:1050B100901DBFE0FF120026D2CA22E4F542C2CA07
:0350C100C20E22FA
:1065D600900028E0FF6026200E07124CF275281462
:1065E60022E528D394004003152822202608D2CA83
:0E65F600752814D22622C2CA75287DC226221C
:10657800200E0C7F1C124CF275286475793C22E5BC
:1065880028D394004003152822AF791579D3EF64F6
:0E659800809480400475286422C20EE4F5420F
:0165A60022D2
:10627B00E54214601C14601C14601F14602214602F
:10628B002224057021C2CAC20EC226C21CE4F544E8
:10629B00220250411265D6D21D2212408CD21D22F1
:0762AB000265781250C422C5
:1063BF00BF010790002A7418F022BF020790002A2D
:1063CF007412F022BF030590002A8014BF040790B7
:1063DF00002A740BF02290002ABF05047409F022E2
:0463EF00740CF02218
:024FBB00AC0741
:104FBD00C3EC64809480404AEC6480948850432014
:104FCD002A21E4FD124CFCC333CE33CED8F9124C5A
:104FDD007774102BF58274003AF583EFF00DBD0850
:104FED00E3801FE4FD124CFCC333CE33CED8F9124F
:104FFD004C7774182BF58274003AF583EFF00DBDE4
:10500D0008E3202A16E4FDEDFF3395E0FE74102F22
:10501D00F5827400124CA8BD08ED22302A15E4FD6E
:10502D00EDFF3395E0FE74182FF5827400124CA835
:03503D00BD08EDBE
:01504000224D
:105399007D3F7F0912665E7D507F0812665E906EC2
:1053A900F91254007D5B7F0612665E906EFA125404
:1053B90000906EFBE493FDE4FF12665E906EFCE4E0
:1053C9009324BE601414601514601814601B1460D3
:1053D9001E240570217D0A80067D3280027D467F6C
:1053E9000280107D0A7F03800A7D287F0380047D67
:1053F900467F0312665E22E493FDE4FF12665E2295
:105EC2008F5BE55B7005D22CFF8009E55BB40107AF
:105ED200D22C7F011259927D4B7F0212665E7D02A7
:105EE200E4FF12665E7D32E4FF12665E125399E5AC
:105EF2005B70028005E55BB401057F40126E89226A
:103D2E00A209300501B350307D017F04124EAB5015
:103D3E002320050E30090B9000A4E0FF7C0B7D6064
:103D4E00800F30050F20090C9000A5E0FF7C0B7D45
:103D5E0080125BB3A2099205A20A300601B350305D
:103D6E007D027F04124EAB502320060E300A0B90BC
:103D7E0000A6E0FF7C0B7DA0800F30060F200A0C02
:103D8E009000A7E0FF7C0B7DC0125BB3A20A9206E7
:103D9E00A20B300701B350307D037F04124EAB509F
:103DAE002320070E300B0B9000A8E0FF7C0B7DE06C
:103DBE00800F30070F200B0C9000A9E0FF7C0C7DCC
:103DCE0000125BB3A20B9207A20D300801B3503064
:103DDE007D047F04124EAB502320080E300D0B9045
:103DEE0000AAE0FF7C0C7D20800F30080F200D0C08
:103DFE009000ABE0FF7C0C7D40125BB3A20D9208ED
:013E0E002291
:1064B800534103900024E0FE543FFF780408800114
:1064C80023D8FD54F0FFEE30E40343070490002482
:0F64D800E030E503430708EF4241C2AF124C9991
:0164E7002292
:022995008F6B46
:10299700302E05756CF48003756C64E56B6401700B
:1029A70029AF417803EF08800123D8FD33922F7FA9
:1029B70010202F0B122AB17F10126EBD022AA91206
:1029C7002ABC7F10126ED0022AA9E56B6402702818
:1029D700AF417802EF08800123D8FD33922F7F2083
:1029E700202F0A122AB17F20126EBD8008122ABC3E
:1029F7007F20126ED0022AA9E56B64037028AF41CD
:102A07007801EF08800123D8FD33922F7F40202FD4
:102A17000A122AC77F40126EBD8008122AD27F4051
:102A2700126ED0022AA9E56B6404701EE541339249
:102A37002F7F80202F0A122AC77F80126EBD800841
:102A4700122AD27F80126ED08058E56B64057027FA
:102A5700AF417805EF08800123D8FD33922F7F041B
:102A6700202F0A122ADD7F04126EBD8008122AE881
:102A77007F04126ED0802BE56B6406702CAF417813
:102A870004EF08800123D8FD33922F7F08202F0AF7
:102A9700122ADD7F08126EBD8008122AE87F08120D
:092AA7006ED0AF6C7E00126BFFD3
:102AB00022126ED0AF6C7E00126BFF22126EBDAF81
:102AC0006C7E00126BFF22126ED0AF6C7E00126B18
:102AD000FF22126EBDAF6C7E00126BFF22126ED011
:102AE000AF6C7E00126BFF22126EBDAF6C7E0012C7
:032AF0006BFF2257
:105D2600900024E030E0057F10126ED0900024E051
:105D360030E1057F20126ED0900024E030E2057F2E
:105D460040126ED0900024E030E3057F80126ED0C2
:105D5600900024E030E4057F04126ED0900024E029
:095D660030E5057F08126ED02221
:106C500030030A124CDDC203C210C21D22300409E7
:0A6C6000124CDDC204C212C21D2254
:1064E8008F708D71E570B4011FE5717003125C49FE
:1064F800E571B401077880E6FF125A35E571B432C8
:106508000E7FF47E01026BFFAD71AF7012665E22E2
:10665E00EFFEEDFF1280008E2D8F2E1253247574D7
:10666E0032AF741574EFD39400400EE4F573E573F6
:09667E00C3943A50EC057380F559
:0166870022F0
:10532400D2A8AFA875A881C213852E82852D83E4E7
:1053340093C4540FFE4306F08E80C284D28500C20B
:10534400870000D287007580FF7580FEC284C28505
:1053540000C2870000D287007580FFD2137D407C95
:105364001FE4FE30B40D0EBE32F9ED1D70011CEDCC
:105374004C70EE7C1F7D40E4FE20B40D0EBE32F96D
:10538400ED1D70011CED4C70EE8FA8C2A87F0A7E43
:0453940000126BFF99
:0153980022F2
:106688007580FDC284C28500C28700000000D287E1
:10669800007580FF7F0A7E00126BFF7F997E0912CA
:0A66A80080008E2D8F2E1253242245
:10414D00D284D285C286A2809216A281921FA282AB
:10415D009217A2839220D2862001537D027F0112F5
:10416D004EAB40137D037F01124EAB400A30160754
:10417D00301832D22380377D027F01124EAB500FA3
:10418D0030160C301F09301804D223802180167D83
:10419D00037F01124EAB5012201603301F0C301846
:1041AD0004D22380091267558004C218C22320024D
:1041BD004E7D027F02124EAB40127D037F02124EE6
:1041CD00AB4009301706301A2FD224227D027F0210
:1041DD00124EAB500E30170B302008301A03D2247C
:1041ED002280157D037F02124EAB500F2017033036
:1041FD002009301A03D2242202677DC21AC224225A
:10675500753D1E753E60E4FFE53E2FF582E4353D4F
:10676500F583E4F00FBF50F0753D1E753E60E4F50E
:0767750045C225C210D21835
:01677C0022FA
:10677D00753F1E7540B0E4FFE5402FF582E4353FCF
:10678D00F583E4F00FBF10F0753F1E7540B0E4F5D2
:07679D0046C227C212D21A06
:0167A40022D2
:106BA900C284D285C286A2809209A281920AA28257
:0D6BB900920BA283920DD286D284D2852247
:1060EB00E57E2560F582E4357DF5832274FF123B56
:1060FB001AE4FBFAF9F8C3023B07057F7480257E8F
:10610B00F57EE4357DF57D22F582E4341DF58322A1
:0B611B00757F01757D00757E20E42279
:10420D007D027F07124EAB50057F04126EBDC22892
:10421D00D222E4F5427FE87E03126BFFC298C2AF53
:10422D00C22F7F0312300A755E7F755D96755C989F
:10423D00755B00785B1260F7504430983E120006B3
:10424D00126DE0EF14601824F0602624C1600B2479
:10425D00F670287F06126EE2802112619B801C7F12
:10426D0006126EE21269871264B8125DB7D2288009
:10427D000A7F06126EE21259E5D2283028B5E4788D
:10428D0085F6D22F7F0112300A7F40120016C22E02
:10429D001269417D467F0212665E7D1E7F071266A2
:1042AD005E7D147F0812665E7D327F0312665EC2EC
:0D42BD002F7F0312300A7FFF126E89C2228C
:0142CA0022D1
:1059E50012611BF55F7F02126EE2E57F2402F5610D
:1059F500AF7F126EE2E4F5601260EBE0FF126EE23B
:105A05001260EBE02561F5610560E560C3948040B7
:105A1500E7AF61126EE27F03126EE2126EEAEF6487
:0F5A250015600C126105055FE55FC3942240B662
:015A3400224F
:1069870012611BF55F1266DB50077F06126EE2800D
:10699700057F15026EE2126105055FE55FC394226C
:0269A70040E3CB
:0169A90022CB
:1066DB00E4F560126EEA74D02560126113EFF005D9
:1066EB0060E560C3948440EB126DBE901E52E0B522
:0866FB000705126C1AD322C33B
:016703002273
:106C1A00E4FF74D22FF582E4341DF583E0FEE57EAD
:0A6C2A002F1260EFEEF00FBF7FE8BD
:016C3400223D
:106DBE00E4FFFE74D02E126113E02FFF0EBE82F39D
:016DCE0022A2
:10619B00E4F55FF5657564E0756393756204F5610D
:1061AB0078611260F750213098F61200068F60E587
:1061BB006064046013AF65056574D02F126113E53D
:0861CB0060F0255FF55F80D84C
:0161D30022A9
:04000600AF99C29854
:01000A0022D3
:086EE2003099FDC2998F99223D
:076EEA003098FDAF99C2983A
:016EF100227E
:106CB6000C0102030405060708090A0B0C0102036E
:086CC6000405060708090A0B8A
:10670400AF5FEF3395E0FE75F007EF123B38EE759F
:10671400F007A42583F583E0227883E6FF126C84D6
:09672400EF22C295D297D2AF22F8
:10681A00C22BC2AF126EF27F83126CCE126AB8120A
:10682A0067267884E66F600B125E3F302A05125F96
:05683A0002922BA22BCD
:01683F002236
:105F02007984E778876660367884E6FF7887F6EFEB
:105F12007013E552C3940A500C7D077F04124EABF6
:105F22005003125DFC7D057F04124EAB5010E5411B
:105F320054036005123EEFD322123EEFC322C32266
:103EEF00E4F55F900A501267047003023FB3900A23
:103EFF005112670B60167881666003023FB3900A18
:103F0F00521267047888666003023FB3AF5FEF33E6
:103F1F0095E0FE900A5312670BFF7880E6FEEF6E76
:103F2F006020EF601DB4080BEED394014005EE94B2
:103F3F0007400FEF6409706CEE64016005EE6407D3
:103F4F007062AF5FEF3395E0FE900A5412670BFF7C
:103F5F00F46006EF788366704BE55FFD3395E0FC08
:103F6F00900A5575F007ED123B38EC126713788401
:103F7F00667031D201D20274BD2DF58274003CF50A
:103F8F0083E0FFC007EDAE047805C333CE33CED840
:103F9F00F92480F582740E3EAD82FCD007125BB31C
:103FAF00C201C202055FC3E55F64809493500302B0
:023FBF003EF2D0
:013FC10022DD
:105DFC007D087F04124EAB500D7883E6FF126C8445
:105E0C00EFC39407402CD22F7F0112300A7F40122F
:105E1C000016C22E126941D201D202E4FD7F0A1291
:105E2C004F33C201C2027F50126E89C22F7F011202
:035E3C00300A2207
:105E3F00C2AF126EF27FBF126CCE126AB87884A610
:105E4F0007126AB87884A607126AB87883A6071271
:105E5F006AB87888A607126AB87881A607126AB856
:105E6F007880A607126AB87882A607126EF21267B8
:025E7F002622D9
:10577E00C2AF126EF27F8E1257CD7F90126CCE7F1B
:10578E00A7126CCE126EF27FBE126CCEE4FF126CBC
:10579E00CE7884E6FF126CCE7883E6FF126CCE785C
:1057AE0088E6FF126CCE7881E6FF126CCE7880E62A
:1057BE00FF126CCE7882E6FF1257CD1267262212A8
:0B57CE006CCEE4FF126CCE126EF222D3
:105A35008F72E572B401047D63803EE572B402069F
:105A45007D087F068035E572B403067D317F0880C9
:105A55002AE572B404067D617F08801FE572B405EE
:105A6500067D257F088014E572B406067D597F03FF
:0F5A75008009E572B407077D487F0712665E223D
:026C8400AE0759
:106C8600EE54F0FF780408800103D8FD75F00AA4DD
:066C9600FFEE540F2FFF7A
:016C9C0022D5
:105C490012671D906CB693FF1234C5788412671FD2
:105C5900601B788412671FC3940A50077D327F0640
:105C690012665E7884E6FF126C841234C512671DD1
:105C7900C3940C50067D0A7F0280047D507F061272
:0A5C8900665E7D507F0512665E2204
:10593C007FF47E01126BFF7D097F0612665E788113
:10594C001259827D0E7F0312665E7D357F061266CC
:10595C005E7D097F0612665E78881259827D1E7FF5
:10596C000912665E7D1E7F0712665E7882E6FF1264
:10597C006C841234C522E6FF126C841234C57FF499
:06598C007E01126BFF22F8
:076EF200C2B6C295D2952241
:106CCE00E4FEC297EF30E002D297C2B6D2B6EFC35F
:066CDE0013FF0EBE08ECDE
:016CE400228D
:106AB800E4FFD297FED2B6C2B6A297E433C433330A
:0F6AC800335480FDEFC313FFED42070EBE08E607
:016AD700229C
:1056C600EF3395E0FE74702FF58274003EF583E0AB
:1056D600FF22AF5AEF3395E0FEEF222460F5827485
:1056E600013EAD82FCD22822900520E0F547A3E0DA
:1056F600F548222450F58274053EAD82FC229000C6
:10570600BAE0FF7C0E7D2022D221D201E4FF22C224
:0D57160001C2217F1922D221D22F7F022251
:10283400E5527008126C9D8F5202292FE552B4059F
:10284400081245A88F5202292FE552B40B08126DC5
:10285400288F5202292FE552B40A08125C938F5232
:1028640002292FE552B40F08125FFB8F5202292F61
:10287400E552B4140812234D8F5202292FE552B4A5
:102884001908126B158F5202292FE552B41E081233
:1028940069F08F5202292FE552B42308126A568F29
:1028A4005202292FE552B42807126E978F52807B6B
:1028B400E552B42D071267CD8F52806FE552B432C2
:1028C400071261D48F528063E552B43E07126B3312
:1028D4008F528057E552B43C07126D888F52804B5B
:1028E400E552B43307126A348F52803FE552B44143
:1028F40007126E118F528033E552B44C07126E21C9
:102904008F528027E552B44407126E318F52801BD8
:10291400E552B437071258338F52800FE552B43959
:10292400071257D98F528003E4F552E5537006120B
:10293400000E8F5322E553B40506126ED98F53222D
:10294400E553B40A06126E418F5322E553B40F06C1
:10295400126E508F5322E553B41406123B6A8F5300
:1029640022E553B43D06126B518F5322E553B43F15
:10297400061265188F5322E553B443061267A58FD8
:102984005322E553B44D06126A778F5322E4F5536C
:012994002220
:106C9D007D077F05124EAB500D30000A90052AE09E
:096CAD00F52BA3E0F52C7F052274
:1045A800302314200F11C21B7D047F01124EAB5023
:1045B800037F0B227F0A227F081262B25006124440
:1045C800F37F0022202308300F05C20F7F05227DCC
:1045D800057F06124EAB501EE5394538701890001D
:1045E800B5E0FF7C0D7D80125BB390052EE0F538B9
:1045F800A3E0F53980487D067F06124EAB501EE5D4
:104608003C453B70189000B6E0FF7C0D7DA0125B26
:10461800B3900530E0F53BA3E0F53C80217D077FB2
:1046280005124EAB500D30000AE52C452B7004C224
:1046380000800B7885E6B405057F04125142E551E8
:0D464800700875510AD22A12681A7F0522E7
:106D280090053BE0F54E2023037F0522E54ED394E2
:066D38000050F37F0A2267
:105C93007D077F05124EAB500C7D077F05124EAB7F
:105CA300503230002F7D017F01124EAB5026D22F90
:105CB3007F0112300A7F011200167D027F07124E08
:105CC300AB50057F04126ED09000A0E0FF7C0A7DEC
:0A5CD300E0125BB31256EE7F0F22C1
:105FFB00302337E5484547700C7D087F01124EABC7
:10600B0050037F372230030EE53A700A126C507F33
:10601B000112001680113025037F14227885E6B417
:0D602B0005057F031251427F0F227F1422D2
:10234D0090053DE0F54B7F01126E89126C507D02B8
:10235D007F07124EAB5009E54B70057F04126EBD21
:10236D009000A1E0FF7C0B7D00125BB3D22A1268B6
:10237D001AE54570030224777C017D001224F55087
:10238D00037F3E227C017D501224D550037F3C22D9
:10239D007C017D581224D550037F3C227C017D1099
:1023AD001224DD50081224E550037F33227C017D79
:1023BD00201224DD500B9000BBE0FF7C0E7D408091
:1023CD00207C017D281224ED500512570480127CCB
:1023DD00017D301224ED50129000B9E0FF7C0E7D8E
:1023ED0000125BB31267557F00227C017D40D2281D
:1023FD00E4FF1247AB500C7D067F04124EAB500329
:10240D007F4C227C017D381224F550037F44227CC1
:10241D00017D18C228E4FF1247AB500C7D057F01EA
:10242D00124EAB50037F4122E4F55A1256D8780371
:10243D00C333CE33CED8F91256E1E4FF1247AB5079
:10244D001BAF5A1256C6C0071256D87805C333CEE5
:10245D0033CED8F91256F9D007125B68055AC3E589
:10246D005A648094A840C47F19221224E5500C7D33
:10247D00077F05124EAB504130003E7885E6700463
:10248D007F0180087885E6B404077F0212514280EF
:10249D00257D037F06124EAB501CE5574556701631
:1024AD009000AFE0FF7C0C7DC0125BB3900532E075
:1024BD00F556A3E0F5577F19227D077F05124EAB28
:0724CD0050052000027F050D
:1024D40022D228E4FF1247AB22D228E4FF1247ABF2
:1024E400227D077F05124EAB22D228E4FF1247ABB0
:0924F40022C228E4FF1247AB22CA
:106B15003025031267557D077F05124EAB500620C1
:0E6B250000037F0522900538E0F54E7F1E220A
:1069F000E54E70037F23227D027F07124EAB5009C4
:106A0000E54B70057F04126EBD3023037F0A227FA1
:026A10001E2244
:106A56001256EE7D067F01124EAB500C9000ACE054
:106A6600FF7C0C7D60125BB3900539E0F54E7F2DFF
:016A760022FD
:0E6E97007FA0126E89900539E0F54E7F2D2206
:1067CD00D22A12681A7D027F07124EAB5009E54B93
:1067DD0070057F04126EBDE54E70037F32223023AB
:0767ED00037F0A227F2D2229
:1061D400301D037F32227D047F06124EAB501FE533
:1061E40055455470199000B0E0FF7C0C7DE0125BC3
:1061F400B3900534E0F554A3E0F5557F3222C22F65
:086204007F0112300A7F002225
:106D880020210CD221E4FF12055BC2217F00227F63
:026D98003C229B
:106B3300202118D2217F40120016D201121D94C2C7
:0E6B4300017F40126E89C2217F19227F3E22FF
:106E110020210A12570E1235C4125715227F412222
:106E210020210A12570E126074125715227F442234
:106E310020210A12570E125475125715227F44222F
:05000E0000007F052247
:096ED9003024037F0A227F052208
:0F6E41009000A2E0FF7C0B7D20125BB37F0F223D
:0F6E50003024093027037F14227F0F227F142262
:103B6A009000A3E0FF7C0B7D40125BB3E546700337
:103B7A00023C427D017F03124EAB50707C017D08EE
:103B8A00C2287F011247AB50037F3F227C017D5040
:103B9A00123C4550037F3D227C017D58123C455022
:103BAA00037F3D227C017D40D2287F011247AB5022
:103BBA000C7D067F04124EAB50037F4D227C017DA3
:103BCA0028D2287F011247AB5009125704125BB35F
:103BDA007F00227C017D18C2287F011247AB500C5E
:103BEA007D057F02124EAB50037F43227D027F0385
:103BFA00124EAB5043E4F55AAF5A1256DA7803C361
:103C0A0033CE33CED8F91256E17F011247AB501D9D
:103C1A00AF5A1256C6C007AF5A1256DA7805C333DE
:103C2A00CE33CED8F91256F9D007125B68055AC3BB
:0A3C3A00E55A648094A840C07F00A2
:093C440022D2287F011247AB22B5
:106B5100202118D221C22F7F0112300A7F01126E2B
:0E6B6100897F0112055BC2217F00227F3D2249
:1065180020212A12571C12300A7FF47E01126BFFC9
:106528007F10120016D202121B93C2027F10126E45
:1065380089C22F7F0212300AC2217F00227F3F22A8
:1067A50020212212571C12300A7FF47E01126BFF42
:1067B500D2027F011235C4C202C22F7F0212300AF3
:0867C500C2217F00227F432264
:106A770020211B12571C12300AD2027F01126074A8
:106A8700C202C22F7F0212300AC2217F00227F4D2D
:016A970022DC
:1055A900AF5AEF3395E0FE22900520E0F547A3E0DE
:1055B900F54822900522E0F549A3E0F54A22246046
:1055C900F58274013EAD82FCD2282274702FF582D7
:1055D90074003EF583E0FF22C202C2217F19222412
:1055E90050F58274053EAD82FC22055AC3E55A6422
:1055F9008094A822D221C22F7F0122D221C22F7FDB
:0256090002227B
:10327100E55270061266048F5222E552B405061219
:1032810038A18F5222E552B40B06126A128F5222D4
:10329100E552B40A061242CB8F5222E552B40F0610
:1032A100126D9A8F5222E552B411061258E48F52D0
:1032B10022E552B412061251BC8F5222E552B414C7
:1032C10006120D3F8F5222E552B419061265A78FDF
:1032D1005222E552B41E061265488F5222E552B4BD
:1032E1002306125E818F5222E552B42806126EA582
:1032F1008F5222E552B42D061261268F5222E552D9
:10330100B4320612620C8F5222E552B43C06126DA1
:10331100AC8F5222E552B43D06126C358F5222E534
:1033210052B43E061268AF8F5222E552B43F0612E4
:103331006DCF8F5222E552B44106126AD88F5222C4
:10334100E552B443061269AA8F5222E552B44C06E3
:10335100126C6A8F5222E552B44D061269CD8F521A
:1033610022E552B437061258338F5222E552B4394E
:10337100061257D98F5222E552B438061268D48FFB
:103381005222E552B43306126A348F5222E552B406
:0C3391004406126CE58F5222E4F5522233
:106604007D077F05124EAB500D30000A90052AE03D
:10661400F52BA3E0F52C7D067F02124EAB500C90B7
:0E662400052CE0F529A3E0F52AD21E7F052201
:1038A100302314200F11C21B7D047F01124EAB5037
:1038B100037F0B227F0A22302414201111D21B7D99
:1038C100047F02124EAB50037F0B227F0A227F0836
:1038D1001262B250061244F37F0022202308300FF7
:1038E10005C20F7F0522202408301105C2117F0572
:1038F100227D057F06124EAB501EE5394538701802
:103901009000B5E0FF7C0D7D80125BB390052EE049
:10391100F538A3E0F53980687D067F06124EAB507D
:103921001EE53C453B70189000B6E0FF7C0D7DA084
:10393100125BB3900530E0F53BA3E0F53C80417D9F
:10394100077F05124EAB500B300008E52C452B705C
:1039510002C2007D067F02124EAB5019301E16E5E1
:103961002A45297010C21E9000BCE0FF7C0E7D60CC
:10397100125BB3800B7885E6B405057F04125142D2
:0F398100E551700875510AD22A12681A7F052283
:106A120090053BE0F54E202306201B037F05222034
:106A22002406301B037F0522E54ED3940050E77FF6
:026A32000A2236
:1042CB007D077F05124EAB50127D077F05124EAB5B
:1042DB00400302437C20000302437C201B3FD22F70
:1042EB007F0312300A7F0F126E8990000FE0B40229
:1042FB00047F05800990000FE0B403057F011200D5
:10430B00161255B17D027F07124EAB50057F04127A
:10431B006ED09000A0E0FF7C0A7DE0804E301B51F8
:10432B0090000FE0FF64026005EF640370437F0FA2
:10433B00126E897F051262B2400BD22F7F011230B1
:10434B000A7F028009D22F7F0312300A7F0A1200E4
:10435B00167D027F07124EAB50057F04126ED012F2
:10436B0055BC9000A2E0FF7C0B7D20125BB37F0F4E
:0A437B00221255B11255BC7F0F222B
:106D9A00201B063023037F1122301B053024027F7B
:026DAA001222B3
:1058E400302352E5484547700C7D087F01124EABCA
:1058F40050037F3722300329E53A70257FA0126ECA
:105904008990000FE0B401047F01800990000FE04A
:10591400B402057F05120016E4F542C21DC20380DD
:10592400113025037F14227885E6B405057F031220
:0859340051427F11227F142271
:1051BC00301B1030230D200F0A7F0A126E89C21B80
:1051CC007F0A22301B4C3024492011463003031235
:1051DC006C50E54A4549700C7D087F02124EAB506D
:1051EC00037F3822300417E53A70137FA0126E89C2
:1051FC007F02120016E4F542C21DC2048011302752
:10520C00037F14227885E6B405057F031251427F93
:10521C001222201B1230240F20110CD21BC22F7F04
:0A522C000212300A7F0A227F1422CA
:100D3F0090053DE0F54B7F0F126E89201B0C900044
:100D4F00A1E0FF7C0B7D00125BB3301B0C9000A366
:100D5F00E0FF7C0B7D40125BB3E542B403037F14CD
:100D6F0022126C50E4F5427D027F07124EAB500900
:100D7F00E54B70057F04126EBDD22A12681A301B24
:100D8F0003020E82E5457003020E827C017D001284
:100D9F000FFF50037F3E227C017D50120FCF500377
:100DAF007F3C227C017D58120FCF50037F3C227C69
:100DBF00017D10120FD75008120FE750037F332217
:100DCF007C017D20120FD75003020EE97C017D2894
:100DDF00120FEF500C9000BAE0FF7C0E7D20020E38
:100DEF00F27C017D30120FEF500C9000B9E0FF7CC8
:100DFF000E7D00020EF27C017D40D228E4FF1247E7
:100E0F00AB500C7D067F04124EAB50037F4C227CFF
:100E1F00017D38120FFF50037F44227C017D18C2E1
:100E2F0028E4FF1247AB500C7D057F01124EAB50EB
:100E3F00037F4122E4F55A1255A9EF7803C333CE4D
:100E4F0033CED8F91255C7E4FF1247AB501D1255D8
:100E5F00A91255D4C0071255A9EF7805C333CE3365
:100E6F00CED8F91255E8D007125B681255F340C778
:100E7F007F1922201B03020F75E5467003020F75C1
:100E8F007D017F03124EAB4003020F2D7C017D08C5
:100E9F00C2287F011247AB500F7F50120016D22F7E
:100EAF007F0212300A7F3F227C017D50120FDF50EC
:100EBF00037F3D227C017D58120FDF50037F3D22BF
:100ECF007C017D10120FF75008120FE750037F338C
:100EDF00227C017D20120FF750129000BBE0FF7CA7
:100EEF000E7D40125BB31267557F00227C017D405F
:100EFF00D2287F011247AB500C7D067F04124EABF8
:100F0F0050037F4D227C017D18C2287F011247AB11
:100F1F00500C7D057F02124EAB50037F43227D02A2
:100F2F007F03124EAB503CE4F55A1255A9EF7803EC
:100F3F00C333CE33CED8F91255C77F011247AB500A
:100F4F001D1255A91255D4C0071255A9EF7805C324
:100F5F0033CE33CED8F91255E8D007125B6812554D
:100F6F00F340C77F19221210075008121007504183
:100F7F0030003E7885E670047F0180087885E6B4FE
:100F8F0004077F0212514280257D037F06124EAB6C
:100F9F00501CE557455670169000AFE0FF7C0C7D56
:100FAF00C0125BB3900532E0F556A3E0F5577F19F9
:0F0FBF00227D077F05124EAB50052000027F05F3
:100FCE0022D228E4FF1247AB22D228E4FF1247AB0D
:100FDE0022D2287F011247AB227D077F05124EAB2E
:100FEE0022D228E4FF1247AB22D2287F011247AB50
:100FFE0022C228E4FF1247AB227D077F05124EABBB
:01100E0022BF
:1065A700C218C22F7F0212300A30250512675580A4
:1065B7000630270312677D7D077F05124EAB500615
:0F65C7002000037F0522900538E0F54E7F1E224D
:10654800E54E70037F23227D027F07124EAB500970
:10655800E54B70057F04126EBD302306200F037FC4
:106568000A22302408201105D21B7F0A227F1E220E
:105E8100201B051255B180031255BC7D067F0112FE
:105E91004EAB5024E5427020201B0B9000ACE0FF7C
:105EA1007C0C7D60800C301B0C9000ADE0FF7C0C05
:105EB1007D80125BB37F2822900539E0F54E7F2D5E
:015EC10022BE
:0E6EA5007FA0126E89900539E0F54E7F2D22F8
:10612600D22A12681A7D027F07124EAB5009E54B40
:1061360070057F04126EBDE54E601D302306200FEC
:10614600037F0A2290000FE06401600930240620D4
:0B61560011037F05227F2D227F3222E3
:10620C00301D037F32227D047F06124EAB501FE5FA
:10621C0055455470199000B0E0FF7C0C7DE0125B8A
:10622C00B3900534E0F554A3E0F5557F3222C22F2C
:08623C007F0112300A7F0022ED
:106DAC0020210CD221E4FF12055BC2217F00227F3F
:026DBC003C2277
:1068AF0020211FC22F7F0212300AD2217F401200F7
:1068BF0016D201121D94C2017F40126E89C2217F30
:0568CF0019227F3E22AA
:106DCF0020210BD221D202121B931255E1227F3FB9
:016DDF002291
:106C35002021151255FD12300A7F40126E897F0101
:0B6C450012055BC2217F00227F3D2270
:106AD80020211912560412300A7F10126E89D20131
:0F6AE800E4FF1235C4C201C2217F19227F41226F
:1069AA0020211D1255FD12300A7F40126E89D22F06
:1069BA007F0212300AD2027F011235C41255E12237
:0369CA007F4322E6
:106C6A0020211412560412300AD201E4FF12607471
:0A6C7A00C201C2217F19227F4122CE
:1069CD0020211D1255FD12300A7F40126E89D22FE3
:1069DD007F0212300AD2027F011260741255E12239
:0369ED007F4322C3
:106CE50020211112560412300AD202E4FF12547503
:076CF5001255E1227F442249
:10583300D20F7D027F07124EAB50057F04126EBD5F
:1058430090000FE0FF64016004EFB4030E7F0112C8
:105853006E897F4012587C7F01801390000FE0B463
:10586300020F7F05126E897F5012587C7F03126EE0
:10587300BD7F50126E897F3922120016C22E126923
:0958830041E4FD7F07124F3322BE
:1057D9003023037F3922E47885F6C20F90000FE069
:1057E900FF64016004EFB4030E7F01126ED07F40A5
:1057F9001258237F01801890000FE0B402147F0330
:10580900126ED07F05126E897F501258237F0312C2
:105819006EBD7F50126E897F0022120016C22E12B1
:0A5829006941E4FD7F08124F3322AD
:1068D400D2117F0A126E897F40120016D22E1269DD
:1068E40041E4FD7F07124F337F03126EBD7F5012C8
:0568F4006E897F002207
:106A340030000B9000B8E0FF7C0D7DE0800C20005E
:106A44000E9000B7E0FF7C0D7DC0125BB3B2007FF7
:026A5400192205
:106074008F5AE55A24FF922E126941E55A70127F15
:1060840040120016D201E4FD7F09124F33C2018091
:1060940015E55AB401107F10120016D202E4FD7FF8
:0C60A40009124F33C2027F50126E892295
:104D9300C201C202D20C7F50126E897F80120016AC
:104DA30075420390000FE0B401163023647F0112B3
:104DB3000016302307E542D3940050F67F01804E5E
:104DC30090000FE0FF64026005EF6403704330233B
:104DD300267F02126E89D22F7F0312300A7F0512BB
:104DE3000016302307E542D3940050F6C22F7F020A
:104DF30012300A7F0580173024177F021200163005
:104E0300240AE542D3940040033023F37F02126E59
:0D4E130089E542708E7FA0126E89C20C22CC
:03000000026BC6CA
:106BC600758E0078FEE4F6D8FD9000007FFF7E1FEC
:0D6BD600E4F0A3DFFCDEFA758188024BE7D6
:103A7E00C2D530F707B2D563F0FF05F030E70CB2D0
:103A8E00D5F4048463F0FF05F080018430D502F490
:023A9E00042200
:103AA000EF8DF0A4A8F0CF8CF0A428CE8DF0A42E3A
:023AB000FE22F4
:103AB200BC000BBE0029EF8DF084FFADF022E4CCF8
:103AC200F875F008EF2FFFEE33FEEC33FCEE9DECC1
:103AD200984005FCEE9DFE0FD5F0E9E4CEFD22ED07
:103AE200F8F5F0EE8420D21CFEADF075F008EF2F51
:103AF200FFED33FD4007985006D5F0F222C398FD42
:053B02000FD5F0EA22DE
:103B0700EB9FF5F0EA9E42F0E99D42F0E89C45F014
:013B1700228B
:103B18007401FF3395E0FEFDFC080808E6CF2FF698
:103B280018E6CE3EF618E6CD3DF618E6CC3CF62271
:0C3B3800A42582F582E5F03583F5832298
:103B4400D083D082F8E4937012740193700DA3A310
:103B540093F8740193F5828883E473740293686024
:063B6400EFA3A3A380DF24
:106DE000EFC39461400AEF947B5005EF24E0FF224B
:016DF0002280
:00000001FF
